
05_uart_tx.elf:     file format elf32-littlearm

Sections:
Idx Name          Size      VMA       LMA       File off  Algn
  0 .isr_vector   00000198  08000000  08000000  00010000  2**0
                  CONTENTS, ALLOC, LOAD, READONLY, DATA
  1 .text         000012dc  080001a0  080001a0  000101a0  2**4
                  CONTENTS, ALLOC, LOAD, READONLY, CODE
  2 .rodata       000000a4  0800147c  0800147c  0001147c  2**2
                  CONTENTS, ALLOC, LOAD, READONLY, DATA
  3 .ARM.extab    00000000  08001520  08001520  00020064  2**0
                  CONTENTS
  4 .ARM          00000000  08001520  08001520  00020064  2**0
                  CONTENTS
  5 .preinit_array 00000000  08001520  08001520  00020064  2**0
                  CONTENTS, ALLOC, LOAD, DATA
  6 .init_array   00000004  08001520  08001520  00011520  2**2
                  CONTENTS, ALLOC, LOAD, DATA
  7 .fini_array   00000004  08001524  08001524  00011524  2**2
                  CONTENTS, ALLOC, LOAD, DATA
  8 .data         00000064  20000000  08001528  00020000  2**2
                  CONTENTS, ALLOC, LOAD, DATA
  9 .bss          00000038  20000064  0800158c  00020064  2**2
                  ALLOC
 10 ._user_heap_stack 00000604  2000009c  0800158c  0002009c  2**0
                  ALLOC
 11 .ARM.attributes 00000030  00000000  00000000  00020064  2**0
                  CONTENTS, READONLY
 12 .debug_info   000027e1  00000000  00000000  00020094  2**0
                  CONTENTS, READONLY, DEBUGGING, OCTETS
 13 .debug_abbrev 000006ad  00000000  00000000  00022875  2**0
                  CONTENTS, READONLY, DEBUGGING, OCTETS
 14 .debug_aranges 00000138  00000000  00000000  00022f28  2**3
                  CONTENTS, READONLY, DEBUGGING, OCTETS
 15 .debug_ranges 00000100  00000000  00000000  00023060  2**3
                  CONTENTS, READONLY, DEBUGGING, OCTETS
 16 .debug_macro  0000f787  00000000  00000000  00023160  2**0
                  CONTENTS, READONLY, DEBUGGING, OCTETS
 17 .debug_line   000014d2  00000000  00000000  000328e7  2**0
                  CONTENTS, READONLY, DEBUGGING, OCTETS
 18 .debug_str    00055258  00000000  00000000  00033db9  2**0
                  CONTENTS, READONLY, DEBUGGING, OCTETS
 19 .comment      00000053  00000000  00000000  00089011  2**0
                  CONTENTS, READONLY
 20 .debug_frame  00000bcc  00000000  00000000  00089064  2**2
                  CONTENTS, READONLY, DEBUGGING, OCTETS

Disassembly of section .text:

080001a0 <__do_global_dtors_aux>:
 80001a0:	b510      	push	{r4, lr}
 80001a2:	4c05      	ldr	r4, [pc, #20]	; (80001b8 <__do_global_dtors_aux+0x18>)
 80001a4:	7823      	ldrb	r3, [r4, #0]
 80001a6:	b933      	cbnz	r3, 80001b6 <__do_global_dtors_aux+0x16>
 80001a8:	4b04      	ldr	r3, [pc, #16]	; (80001bc <__do_global_dtors_aux+0x1c>)
 80001aa:	b113      	cbz	r3, 80001b2 <__do_global_dtors_aux+0x12>
 80001ac:	4804      	ldr	r0, [pc, #16]	; (80001c0 <__do_global_dtors_aux+0x20>)
 80001ae:	f3af 8000 	nop.w
 80001b2:	2301      	movs	r3, #1
 80001b4:	7023      	strb	r3, [r4, #0]
 80001b6:	bd10      	pop	{r4, pc}
 80001b8:	20000064 	.word	0x20000064
 80001bc:	00000000 	.word	0x00000000
 80001c0:	08001464 	.word	0x08001464

080001c4 <frame_dummy>:
 80001c4:	b508      	push	{r3, lr}
 80001c6:	4b03      	ldr	r3, [pc, #12]	; (80001d4 <frame_dummy+0x10>)
 80001c8:	b11b      	cbz	r3, 80001d2 <frame_dummy+0xe>
 80001ca:	4903      	ldr	r1, [pc, #12]	; (80001d8 <frame_dummy+0x14>)
 80001cc:	4803      	ldr	r0, [pc, #12]	; (80001dc <frame_dummy+0x18>)
 80001ce:	f3af 8000 	nop.w
 80001d2:	bd08      	pop	{r3, pc}
 80001d4:	00000000 	.word	0x00000000
 80001d8:	20000068 	.word	0x20000068
 80001dc:	08001464 	.word	0x08001464

080001e0 <memchr>:
 80001e0:	f001 01ff 	and.w	r1, r1, #255	; 0xff
 80001e4:	2a10      	cmp	r2, #16
 80001e6:	db2b      	blt.n	8000240 <memchr+0x60>
 80001e8:	f010 0f07 	tst.w	r0, #7
 80001ec:	d008      	beq.n	8000200 <memchr+0x20>
 80001ee:	f810 3b01 	ldrb.w	r3, [r0], #1
 80001f2:	3a01      	subs	r2, #1
 80001f4:	428b      	cmp	r3, r1
 80001f6:	d02d      	beq.n	8000254 <memchr+0x74>
 80001f8:	f010 0f07 	tst.w	r0, #7
 80001fc:	b342      	cbz	r2, 8000250 <memchr+0x70>
 80001fe:	d1f6      	bne.n	80001ee <memchr+0xe>
 8000200:	b4f0      	push	{r4, r5, r6, r7}
 8000202:	ea41 2101 	orr.w	r1, r1, r1, lsl #8
 8000206:	ea41 4101 	orr.w	r1, r1, r1, lsl #16
 800020a:	f022 0407 	bic.w	r4, r2, #7
 800020e:	f07f 0700 	mvns.w	r7, #0
 8000212:	2300      	movs	r3, #0
 8000214:	e8f0 5602 	ldrd	r5, r6, [r0], #8
 8000218:	3c08      	subs	r4, #8
 800021a:	ea85 0501 	eor.w	r5, r5, r1
 800021e:	ea86 0601 	eor.w	r6, r6, r1
 8000222:	fa85 f547 	uadd8	r5, r5, r7
 8000226:	faa3 f587 	sel	r5, r3, r7
 800022a:	fa86 f647 	uadd8	r6, r6, r7
 800022e:	faa5 f687 	sel	r6, r5, r7
 8000232:	b98e      	cbnz	r6, 8000258 <memchr+0x78>
 8000234:	d1ee      	bne.n	8000214 <memchr+0x34>
 8000236:	bcf0      	pop	{r4, r5, r6, r7}
 8000238:	f001 01ff 	and.w	r1, r1, #255	; 0xff
 800023c:	f002 0207 	and.w	r2, r2, #7
 8000240:	b132      	cbz	r2, 8000250 <memchr+0x70>
 8000242:	f810 3b01 	ldrb.w	r3, [r0], #1
 8000246:	3a01      	subs	r2, #1
 8000248:	ea83 0301 	eor.w	r3, r3, r1
 800024c:	b113      	cbz	r3, 8000254 <memchr+0x74>
 800024e:	d1f8      	bne.n	8000242 <memchr+0x62>
 8000250:	2000      	movs	r0, #0
 8000252:	4770      	bx	lr
 8000254:	3801      	subs	r0, #1
 8000256:	4770      	bx	lr
 8000258:	2d00      	cmp	r5, #0
 800025a:	bf06      	itte	eq
 800025c:	4635      	moveq	r5, r6
 800025e:	3803      	subeq	r0, #3
 8000260:	3807      	subne	r0, #7
 8000262:	f015 0f01 	tst.w	r5, #1
 8000266:	d107      	bne.n	8000278 <memchr+0x98>
 8000268:	3001      	adds	r0, #1
 800026a:	f415 7f80 	tst.w	r5, #256	; 0x100
 800026e:	bf02      	ittt	eq
 8000270:	3001      	addeq	r0, #1
 8000272:	f415 3fc0 	tsteq.w	r5, #98304	; 0x18000
 8000276:	3001      	addeq	r0, #1
 8000278:	bcf0      	pop	{r4, r5, r6, r7}
 800027a:	3801      	subs	r0, #1
 800027c:	4770      	bx	lr
 800027e:	bf00      	nop

08000280 <__io_putchar>:
void uart2_tx_init(void);
void uart2_write(int ch);
static void uart_set_baudrate(USART_TypeDef *USARTx, uint32_t PeriphClk, uint32_t BaudRate);
static uint16_t compute_uart_bd(uint32_t PeriphClk, uint32_t BaudRate);

int __io_putchar(int ch){
 8000280:	b580      	push	{r7, lr}
 8000282:	b082      	sub	sp, #8
 8000284:	af00      	add	r7, sp, #0
 8000286:	6078      	str	r0, [r7, #4]
	uart2_write(ch);
 8000288:	6878      	ldr	r0, [r7, #4]
 800028a:	f000 f859 	bl	8000340 <uart2_write>
	return ch;
 800028e:	687b      	ldr	r3, [r7, #4]
}
 8000290:	4618      	mov	r0, r3
 8000292:	3708      	adds	r7, #8
 8000294:	46bd      	mov	sp, r7
 8000296:	bd80      	pop	{r7, pc}

08000298 <main>:

int main(void){
 8000298:	b580      	push	{r7, lr}
 800029a:	af00      	add	r7, sp, #0
	uart2_tx_init();
 800029c:	f000 f806 	bl	80002ac <uart2_tx_init>
	while (1){
		printf("hello.. \n\r");
 80002a0:	4801      	ldr	r0, [pc, #4]	; (80002a8 <main+0x10>)
 80002a2:	f000 f989 	bl	80005b8 <iprintf>
 80002a6:	e7fb      	b.n	80002a0 <main+0x8>
 80002a8:	0800147c 	.word	0x0800147c

080002ac <uart2_tx_init>:
	}
}

void uart2_tx_init(void){
 80002ac:	b580      	push	{r7, lr}
 80002ae:	af00      	add	r7, sp, #0
	/*********configure the uart gpioa pin*********/
	/*enable clock access to gpioa*/
	RCC->AHB1ENR |= GPIOAEN;
 80002b0:	4b1f      	ldr	r3, [pc, #124]	; (8000330 <uart2_tx_init+0x84>)
 80002b2:	6b1b      	ldr	r3, [r3, #48]	; 0x30
 80002b4:	4a1e      	ldr	r2, [pc, #120]	; (8000330 <uart2_tx_init+0x84>)
 80002b6:	f043 0301 	orr.w	r3, r3, #1
 80002ba:	6313      	str	r3, [r2, #48]	; 0x30

	/*set PA2 mode to alternate function mode*/
	GPIOA->MODER |= (1U<<5);
 80002bc:	4b1d      	ldr	r3, [pc, #116]	; (8000334 <uart2_tx_init+0x88>)
 80002be:	681b      	ldr	r3, [r3, #0]
 80002c0:	4a1c      	ldr	r2, [pc, #112]	; (8000334 <uart2_tx_init+0x88>)
 80002c2:	f043 0320 	orr.w	r3, r3, #32
 80002c6:	6013      	str	r3, [r2, #0]
	GPIOA->MODER &=~ (1U<<4);
 80002c8:	4b1a      	ldr	r3, [pc, #104]	; (8000334 <uart2_tx_init+0x88>)
 80002ca:	681b      	ldr	r3, [r3, #0]
 80002cc:	4a19      	ldr	r2, [pc, #100]	; (8000334 <uart2_tx_init+0x88>)
 80002ce:	f023 0310 	bic.w	r3, r3, #16
 80002d2:	6013      	str	r3, [r2, #0]

	/*set PA2 alternate function type to UART_TX (AF07)*/
	GPIOA->AFR[0] |= (1U<<8);
 80002d4:	4b17      	ldr	r3, [pc, #92]	; (8000334 <uart2_tx_init+0x88>)
 80002d6:	6a1b      	ldr	r3, [r3, #32]
 80002d8:	4a16      	ldr	r2, [pc, #88]	; (8000334 <uart2_tx_init+0x88>)
 80002da:	f443 7380 	orr.w	r3, r3, #256	; 0x100
 80002de:	6213      	str	r3, [r2, #32]
	GPIOA->AFR[0] |= (1U<<9);
 80002e0:	4b14      	ldr	r3, [pc, #80]	; (8000334 <uart2_tx_init+0x88>)
 80002e2:	6a1b      	ldr	r3, [r3, #32]
 80002e4:	4a13      	ldr	r2, [pc, #76]	; (8000334 <uart2_tx_init+0x88>)
 80002e6:	f443 7300 	orr.w	r3, r3, #512	; 0x200
 80002ea:	6213      	str	r3, [r2, #32]
	GPIOA->AFR[0] |= (1U<<10);
 80002ec:	4b11      	ldr	r3, [pc, #68]	; (8000334 <uart2_tx_init+0x88>)
 80002ee:	6a1b      	ldr	r3, [r3, #32]
 80002f0:	4a10      	ldr	r2, [pc, #64]	; (8000334 <uart2_tx_init+0x88>)
 80002f2:	f443 6380 	orr.w	r3, r3, #1024	; 0x400
 80002f6:	6213      	str	r3, [r2, #32]
	GPIOA->AFR[0] &=~ (1U<<11);
 80002f8:	4b0e      	ldr	r3, [pc, #56]	; (8000334 <uart2_tx_init+0x88>)
 80002fa:	6a1b      	ldr	r3, [r3, #32]
 80002fc:	4a0d      	ldr	r2, [pc, #52]	; (8000334 <uart2_tx_init+0x88>)
 80002fe:	f423 6300 	bic.w	r3, r3, #2048	; 0x800
 8000302:	6213      	str	r3, [r2, #32]

	/*********configure the uart module *********/
	/*enable clock access to uart2*/
	RCC->APB1ENR |= UART2EN;
 8000304:	4b0a      	ldr	r3, [pc, #40]	; (8000330 <uart2_tx_init+0x84>)
 8000306:	6c1b      	ldr	r3, [r3, #64]	; 0x40
 8000308:	4a09      	ldr	r2, [pc, #36]	; (8000330 <uart2_tx_init+0x84>)
 800030a:	f443 3300 	orr.w	r3, r3, #131072	; 0x20000
 800030e:	6413      	str	r3, [r2, #64]	; 0x40

	/*configure baudrate*/
	uart_set_baudrate(USART2, APB1_CLK, UART_BAUDRATE);
 8000310:	f44f 32e1 	mov.w	r2, #115200	; 0x1c200
 8000314:	4908      	ldr	r1, [pc, #32]	; (8000338 <uart2_tx_init+0x8c>)
 8000316:	4809      	ldr	r0, [pc, #36]	; (800033c <uart2_tx_init+0x90>)
 8000318:	f000 f82a 	bl	8000370 <uart_set_baudrate>

	/*configure the transfer direction*/
	USART2 ->CR1 = CR1_TE;
 800031c:	4b07      	ldr	r3, [pc, #28]	; (800033c <uart2_tx_init+0x90>)
 800031e:	2208      	movs	r2, #8
 8000320:	60da      	str	r2, [r3, #12]

	/*enable uart module*/
	USART2 ->CR1 = CR1_UE;
 8000322:	4b06      	ldr	r3, [pc, #24]	; (800033c <uart2_tx_init+0x90>)
 8000324:	f44f 5200 	mov.w	r2, #8192	; 0x2000
 8000328:	60da      	str	r2, [r3, #12]

}
 800032a:	bf00      	nop
 800032c:	bd80      	pop	{r7, pc}
 800032e:	bf00      	nop
 8000330:	40023800 	.word	0x40023800
 8000334:	40020000 	.word	0x40020000
 8000338:	00f42400 	.word	0x00f42400
 800033c:	40004400 	.word	0x40004400

08000340 <uart2_write>:

void uart2_write(int ch){
 8000340:	b480      	push	{r7}
 8000342:	b083      	sub	sp, #12
 8000344:	af00      	add	r7, sp, #0
 8000346:	6078      	str	r0, [r7, #4]
	/*make sure the transmit data register is empty*/
	while(!(USART2->SR & SR_TXE)){}
 8000348:	bf00      	nop
 800034a:	4b08      	ldr	r3, [pc, #32]	; (800036c <uart2_write+0x2c>)
 800034c:	681b      	ldr	r3, [r3, #0]
 800034e:	f003 0380 	and.w	r3, r3, #128	; 0x80
 8000352:	2b00      	cmp	r3, #0
 8000354:	d0f9      	beq.n	800034a <uart2_write+0xa>
	/*write to transmit data register*/
	USART2->DR = (ch & 0xFF);
 8000356:	687b      	ldr	r3, [r7, #4]
 8000358:	4a04      	ldr	r2, [pc, #16]	; (800036c <uart2_write+0x2c>)
 800035a:	b2db      	uxtb	r3, r3
 800035c:	6053      	str	r3, [r2, #4]
}
 800035e:	bf00      	nop
 8000360:	370c      	adds	r7, #12
 8000362:	46bd      	mov	sp, r7
 8000364:	f85d 7b04 	ldr.w	r7, [sp], #4
 8000368:	4770      	bx	lr
 800036a:	bf00      	nop
 800036c:	40004400 	.word	0x40004400

08000370 <uart_set_baudrate>:

static void uart_set_baudrate(USART_TypeDef *USARTx, uint32_t PeriphClk, uint32_t BaudRate){
 8000370:	b580      	push	{r7, lr}
 8000372:	b084      	sub	sp, #16
 8000374:	af00      	add	r7, sp, #0
 8000376:	60f8      	str	r0, [r7, #12]
 8000378:	60b9      	str	r1, [r7, #8]
 800037a:	607a      	str	r2, [r7, #4]
	USARTx->BRR = compute_uart_bd(PeriphClk, BaudRate);
 800037c:	6879      	ldr	r1, [r7, #4]
 800037e:	68b8      	ldr	r0, [r7, #8]
 8000380:	f000 f808 	bl	8000394 <compute_uart_bd>
 8000384:	4603      	mov	r3, r0
 8000386:	461a      	mov	r2, r3
 8000388:	68fb      	ldr	r3, [r7, #12]
 800038a:	609a      	str	r2, [r3, #8]
}
 800038c:	bf00      	nop
 800038e:	3710      	adds	r7, #16
 8000390:	46bd      	mov	sp, r7
 8000392:	bd80      	pop	{r7, pc}

08000394 <compute_uart_bd>:

static uint16_t compute_uart_bd(uint32_t PeriphClk, uint32_t BaudRate){
 8000394:	b480      	push	{r7}
 8000396:	b083      	sub	sp, #12
 8000398:	af00      	add	r7, sp, #0
 800039a:	6078      	str	r0, [r7, #4]
 800039c:	6039      	str	r1, [r7, #0]
	return ((PeriphClk + (BaudRate/2U))/BaudRate);
 800039e:	683b      	ldr	r3, [r7, #0]
 80003a0:	085a      	lsrs	r2, r3, #1
 80003a2:	687b      	ldr	r3, [r7, #4]
 80003a4:	441a      	add	r2, r3
 80003a6:	683b      	ldr	r3, [r7, #0]
 80003a8:	fbb2 f3f3 	udiv	r3, r2, r3
 80003ac:	b29b      	uxth	r3, r3
}
 80003ae:	4618      	mov	r0, r3
 80003b0:	370c      	adds	r7, #12
 80003b2:	46bd      	mov	sp, r7
 80003b4:	f85d 7b04 	ldr.w	r7, [sp], #4
 80003b8:	4770      	bx	lr

080003ba <_read>:
	_kill(status, -1);
	while (1) {}		/* Make sure we hang here */
}

__attribute__((weak)) int _read(int file, char *ptr, int len)
{
 80003ba:	b580      	push	{r7, lr}
 80003bc:	b086      	sub	sp, #24
 80003be:	af00      	add	r7, sp, #0
 80003c0:	60f8      	str	r0, [r7, #12]
 80003c2:	60b9      	str	r1, [r7, #8]
 80003c4:	607a      	str	r2, [r7, #4]
	int DataIdx;

	for (DataIdx = 0; DataIdx < len; DataIdx++)
 80003c6:	2300      	movs	r3, #0
 80003c8:	617b      	str	r3, [r7, #20]
 80003ca:	e00a      	b.n	80003e2 <_read+0x28>
	{
		*ptr++ = __io_getchar();
 80003cc:	f3af 8000 	nop.w
 80003d0:	4601      	mov	r1, r0
 80003d2:	68bb      	ldr	r3, [r7, #8]
 80003d4:	1c5a      	adds	r2, r3, #1
 80003d6:	60ba      	str	r2, [r7, #8]
 80003d8:	b2ca      	uxtb	r2, r1
 80003da:	701a      	strb	r2, [r3, #0]
	for (DataIdx = 0; DataIdx < len; DataIdx++)
 80003dc:	697b      	ldr	r3, [r7, #20]
 80003de:	3301      	adds	r3, #1
 80003e0:	617b      	str	r3, [r7, #20]
 80003e2:	697a      	ldr	r2, [r7, #20]
 80003e4:	687b      	ldr	r3, [r7, #4]
 80003e6:	429a      	cmp	r2, r3
 80003e8:	dbf0      	blt.n	80003cc <_read+0x12>
	}

return len;
 80003ea:	687b      	ldr	r3, [r7, #4]
}
 80003ec:	4618      	mov	r0, r3
 80003ee:	3718      	adds	r7, #24
 80003f0:	46bd      	mov	sp, r7
 80003f2:	bd80      	pop	{r7, pc}

080003f4 <_write>:

__attribute__((weak)) int _write(int file, char *ptr, int len)
{
 80003f4:	b580      	push	{r7, lr}
 80003f6:	b086      	sub	sp, #24
 80003f8:	af00      	add	r7, sp, #0
 80003fa:	60f8      	str	r0, [r7, #12]
 80003fc:	60b9      	str	r1, [r7, #8]
 80003fe:	607a      	str	r2, [r7, #4]
	int DataIdx;

	for (DataIdx = 0; DataIdx < len; DataIdx++)
 8000400:	2300      	movs	r3, #0
 8000402:	617b      	str	r3, [r7, #20]
 8000404:	e009      	b.n	800041a <_write+0x26>
	{
		__io_putchar(*ptr++);
 8000406:	68bb      	ldr	r3, [r7, #8]
 8000408:	1c5a      	adds	r2, r3, #1
 800040a:	60ba      	str	r2, [r7, #8]
 800040c:	781b      	ldrb	r3, [r3, #0]
 800040e:	4618      	mov	r0, r3
 8000410:	f7ff ff36 	bl	8000280 <__io_putchar>
	for (DataIdx = 0; DataIdx < len; DataIdx++)
 8000414:	697b      	ldr	r3, [r7, #20]
 8000416:	3301      	adds	r3, #1
 8000418:	617b      	str	r3, [r7, #20]
 800041a:	697a      	ldr	r2, [r7, #20]
 800041c:	687b      	ldr	r3, [r7, #4]
 800041e:	429a      	cmp	r2, r3
 8000420:	dbf1      	blt.n	8000406 <_write+0x12>
	}
	return len;
 8000422:	687b      	ldr	r3, [r7, #4]
}
 8000424:	4618      	mov	r0, r3
 8000426:	3718      	adds	r7, #24
 8000428:	46bd      	mov	sp, r7
 800042a:	bd80      	pop	{r7, pc}

0800042c <_close>:

int _close(int file)
{
 800042c:	b480      	push	{r7}
 800042e:	b083      	sub	sp, #12
 8000430:	af00      	add	r7, sp, #0
 8000432:	6078      	str	r0, [r7, #4]
	return -1;
 8000434:	f04f 33ff 	mov.w	r3, #4294967295
}
 8000438:	4618      	mov	r0, r3
 800043a:	370c      	adds	r7, #12
 800043c:	46bd      	mov	sp, r7
 800043e:	f85d 7b04 	ldr.w	r7, [sp], #4
 8000442:	4770      	bx	lr

08000444 <_fstat>:


int _fstat(int file, struct stat *st)
{
 8000444:	b480      	push	{r7}
 8000446:	b083      	sub	sp, #12
 8000448:	af00      	add	r7, sp, #0
 800044a:	6078      	str	r0, [r7, #4]
 800044c:	6039      	str	r1, [r7, #0]
	st->st_mode = S_IFCHR;
 800044e:	683b      	ldr	r3, [r7, #0]
 8000450:	f44f 5200 	mov.w	r2, #8192	; 0x2000
 8000454:	605a      	str	r2, [r3, #4]
	return 0;
 8000456:	2300      	movs	r3, #0
}
 8000458:	4618      	mov	r0, r3
 800045a:	370c      	adds	r7, #12
 800045c:	46bd      	mov	sp, r7
 800045e:	f85d 7b04 	ldr.w	r7, [sp], #4
 8000462:	4770      	bx	lr

08000464 <_isatty>:

int _isatty(int file)
{
 8000464:	b480      	push	{r7}
 8000466:	b083      	sub	sp, #12
 8000468:	af00      	add	r7, sp, #0
 800046a:	6078      	str	r0, [r7, #4]
	return 1;
 800046c:	2301      	movs	r3, #1
}
 800046e:	4618      	mov	r0, r3
 8000470:	370c      	adds	r7, #12
 8000472:	46bd      	mov	sp, r7
 8000474:	f85d 7b04 	ldr.w	r7, [sp], #4
 8000478:	4770      	bx	lr

0800047a <_lseek>:

int _lseek(int file, int ptr, int dir)
{
 800047a:	b480      	push	{r7}
 800047c:	b085      	sub	sp, #20
 800047e:	af00      	add	r7, sp, #0
 8000480:	60f8      	str	r0, [r7, #12]
 8000482:	60b9      	str	r1, [r7, #8]
 8000484:	607a      	str	r2, [r7, #4]
	return 0;
 8000486:	2300      	movs	r3, #0
}
 8000488:	4618      	mov	r0, r3
 800048a:	3714      	adds	r7, #20
 800048c:	46bd      	mov	sp, r7
 800048e:	f85d 7b04 	ldr.w	r7, [sp], #4
 8000492:	4770      	bx	lr

08000494 <_sbrk>:
 *
 * @param incr Memory size
 * @return Pointer to allocated memory
 */
void *_sbrk(ptrdiff_t incr)
{
 8000494:	b580      	push	{r7, lr}
 8000496:	b086      	sub	sp, #24
 8000498:	af00      	add	r7, sp, #0
 800049a:	6078      	str	r0, [r7, #4]
  extern uint8_t _end; /* Symbol defined in the linker script */
  extern uint8_t _estack; /* Symbol defined in the linker script */
  extern uint32_t _Min_Stack_Size; /* Symbol defined in the linker script */
  const uint32_t stack_limit = (uint32_t)&_estack - (uint32_t)&_Min_Stack_Size;
 800049c:	4a14      	ldr	r2, [pc, #80]	; (80004f0 <_sbrk+0x5c>)
 800049e:	4b15      	ldr	r3, [pc, #84]	; (80004f4 <_sbrk+0x60>)
 80004a0:	1ad3      	subs	r3, r2, r3
 80004a2:	617b      	str	r3, [r7, #20]
  const uint8_t *max_heap = (uint8_t *)stack_limit;
 80004a4:	697b      	ldr	r3, [r7, #20]
 80004a6:	613b      	str	r3, [r7, #16]
  uint8_t *prev_heap_end;

  /* Initialize heap end at first call */
  if (NULL == __sbrk_heap_end)
 80004a8:	4b13      	ldr	r3, [pc, #76]	; (80004f8 <_sbrk+0x64>)
 80004aa:	681b      	ldr	r3, [r3, #0]
 80004ac:	2b00      	cmp	r3, #0
 80004ae:	d102      	bne.n	80004b6 <_sbrk+0x22>
  {
    __sbrk_heap_end = &_end;
 80004b0:	4b11      	ldr	r3, [pc, #68]	; (80004f8 <_sbrk+0x64>)
 80004b2:	4a12      	ldr	r2, [pc, #72]	; (80004fc <_sbrk+0x68>)
 80004b4:	601a      	str	r2, [r3, #0]
  }

  /* Protect heap from growing into the reserved MSP stack */
  if (__sbrk_heap_end + incr > max_heap)
 80004b6:	4b10      	ldr	r3, [pc, #64]	; (80004f8 <_sbrk+0x64>)
 80004b8:	681a      	ldr	r2, [r3, #0]
 80004ba:	687b      	ldr	r3, [r7, #4]
 80004bc:	4413      	add	r3, r2
 80004be:	693a      	ldr	r2, [r7, #16]
 80004c0:	429a      	cmp	r2, r3
 80004c2:	d207      	bcs.n	80004d4 <_sbrk+0x40>
  {
    errno = ENOMEM;
 80004c4:	f000 f846 	bl	8000554 <__errno>
 80004c8:	4603      	mov	r3, r0
 80004ca:	220c      	movs	r2, #12
 80004cc:	601a      	str	r2, [r3, #0]
    return (void *)-1;
 80004ce:	f04f 33ff 	mov.w	r3, #4294967295
 80004d2:	e009      	b.n	80004e8 <_sbrk+0x54>
  }

  prev_heap_end = __sbrk_heap_end;
 80004d4:	4b08      	ldr	r3, [pc, #32]	; (80004f8 <_sbrk+0x64>)
 80004d6:	681b      	ldr	r3, [r3, #0]
 80004d8:	60fb      	str	r3, [r7, #12]
  __sbrk_heap_end += incr;
 80004da:	4b07      	ldr	r3, [pc, #28]	; (80004f8 <_sbrk+0x64>)
 80004dc:	681a      	ldr	r2, [r3, #0]
 80004de:	687b      	ldr	r3, [r7, #4]
 80004e0:	4413      	add	r3, r2
 80004e2:	4a05      	ldr	r2, [pc, #20]	; (80004f8 <_sbrk+0x64>)
 80004e4:	6013      	str	r3, [r2, #0]

  return (void *)prev_heap_end;
 80004e6:	68fb      	ldr	r3, [r7, #12]
}
 80004e8:	4618      	mov	r0, r3
 80004ea:	3718      	adds	r7, #24
 80004ec:	46bd      	mov	sp, r7
 80004ee:	bd80      	pop	{r7, pc}
 80004f0:	20020000 	.word	0x20020000
 80004f4:	00000400 	.word	0x00000400
 80004f8:	20000080 	.word	0x20000080
 80004fc:	200000a0 	.word	0x200000a0

08000500 <Reset_Handler>:

  .section .text.Reset_Handler
  .weak Reset_Handler
  .type Reset_Handler, %function
Reset_Handler:
  ldr   r0, =_estack
 8000500:	480d      	ldr	r0, [pc, #52]	; (8000538 <LoopForever+0x2>)
  mov   sp, r0          /* set stack pointer */
 8000502:	4685      	mov	sp, r0
/* Call the clock system intitialization function.*/
  bl  SystemInit
 8000504:	f3af 8000 	nop.w

/* Copy the data segment initializers from flash to SRAM */
  ldr r0, =_sdata
 8000508:	480c      	ldr	r0, [pc, #48]	; (800053c <LoopForever+0x6>)
  ldr r1, =_edata
 800050a:	490d      	ldr	r1, [pc, #52]	; (8000540 <LoopForever+0xa>)
  ldr r2, =_sidata
 800050c:	4a0d      	ldr	r2, [pc, #52]	; (8000544 <LoopForever+0xe>)
  movs r3, #0
 800050e:	2300      	movs	r3, #0
  b LoopCopyDataInit
 8000510:	e002      	b.n	8000518 <LoopCopyDataInit>

08000512 <CopyDataInit>:

CopyDataInit:
  ldr r4, [r2, r3]
 8000512:	58d4      	ldr	r4, [r2, r3]
  str r4, [r0, r3]
 8000514:	50c4      	str	r4, [r0, r3]
  adds r3, r3, #4
 8000516:	3304      	adds	r3, #4

08000518 <LoopCopyDataInit>:

LoopCopyDataInit:
  adds r4, r0, r3
 8000518:	18c4      	adds	r4, r0, r3
  cmp r4, r1
 800051a:	428c      	cmp	r4, r1
  bcc CopyDataInit
 800051c:	d3f9      	bcc.n	8000512 <CopyDataInit>

/* Zero fill the bss segment. */
  ldr r2, =_sbss
 800051e:	4a0a      	ldr	r2, [pc, #40]	; (8000548 <LoopForever+0x12>)
  ldr r4, =_ebss
 8000520:	4c0a      	ldr	r4, [pc, #40]	; (800054c <LoopForever+0x16>)
  movs r3, #0
 8000522:	2300      	movs	r3, #0
  b LoopFillZerobss
 8000524:	e001      	b.n	800052a <LoopFillZerobss>

08000526 <FillZerobss>:

FillZerobss:
  str  r3, [r2]
 8000526:	6013      	str	r3, [r2, #0]
  adds r2, r2, #4
 8000528:	3204      	adds	r2, #4

0800052a <LoopFillZerobss>:

LoopFillZerobss:
  cmp r2, r4
 800052a:	42a2      	cmp	r2, r4
  bcc FillZerobss
 800052c:	d3fb      	bcc.n	8000526 <FillZerobss>

/* Call static constructors */
  bl __libc_init_array
 800052e:	f000 f817 	bl	8000560 <__libc_init_array>
/* Call the application's entry point.*/
  bl main
 8000532:	f7ff feb1 	bl	8000298 <main>

08000536 <LoopForever>:

LoopForever:
    b LoopForever
 8000536:	e7fe      	b.n	8000536 <LoopForever>
  ldr   r0, =_estack
 8000538:	20020000 	.word	0x20020000
  ldr r0, =_sdata
 800053c:	20000000 	.word	0x20000000
  ldr r1, =_edata
 8000540:	20000064 	.word	0x20000064
  ldr r2, =_sidata
 8000544:	08001528 	.word	0x08001528
  ldr r2, =_sbss
 8000548:	20000064 	.word	0x20000064
  ldr r4, =_ebss
 800054c:	2000009c 	.word	0x2000009c

08000550 <ADC_IRQHandler>:
 * @retval : None
*/
  .section .text.Default_Handler,"ax",%progbits
Default_Handler:
Infinite_Loop:
  b Infinite_Loop
 8000550:	e7fe      	b.n	8000550 <ADC_IRQHandler>
	...

08000554 <__errno>:
 8000554:	4b01      	ldr	r3, [pc, #4]	; (800055c <__errno+0x8>)
 8000556:	6818      	ldr	r0, [r3, #0]
 8000558:	4770      	bx	lr
 800055a:	bf00      	nop
 800055c:	20000000 	.word	0x20000000

08000560 <__libc_init_array>:
 8000560:	b570      	push	{r4, r5, r6, lr}
 8000562:	4d0d      	ldr	r5, [pc, #52]	; (8000598 <__libc_init_array+0x38>)
 8000564:	4c0d      	ldr	r4, [pc, #52]	; (800059c <__libc_init_array+0x3c>)
 8000566:	1b64      	subs	r4, r4, r5
 8000568:	10a4      	asrs	r4, r4, #2
 800056a:	2600      	movs	r6, #0
 800056c:	42a6      	cmp	r6, r4
 800056e:	d109      	bne.n	8000584 <__libc_init_array+0x24>
 8000570:	4d0b      	ldr	r5, [pc, #44]	; (80005a0 <__libc_init_array+0x40>)
 8000572:	4c0c      	ldr	r4, [pc, #48]	; (80005a4 <__libc_init_array+0x44>)
 8000574:	f000 ff76 	bl	8001464 <_init>
 8000578:	1b64      	subs	r4, r4, r5
 800057a:	10a4      	asrs	r4, r4, #2
 800057c:	2600      	movs	r6, #0
 800057e:	42a6      	cmp	r6, r4
 8000580:	d105      	bne.n	800058e <__libc_init_array+0x2e>
 8000582:	bd70      	pop	{r4, r5, r6, pc}
 8000584:	f855 3b04 	ldr.w	r3, [r5], #4
 8000588:	4798      	blx	r3
 800058a:	3601      	adds	r6, #1
 800058c:	e7ee      	b.n	800056c <__libc_init_array+0xc>
 800058e:	f855 3b04 	ldr.w	r3, [r5], #4
 8000592:	4798      	blx	r3
 8000594:	3601      	adds	r6, #1
 8000596:	e7f2      	b.n	800057e <__libc_init_array+0x1e>
 8000598:	08001520 	.word	0x08001520
 800059c:	08001520 	.word	0x08001520
 80005a0:	08001520 	.word	0x08001520
 80005a4:	08001524 	.word	0x08001524

080005a8 <memset>:
 80005a8:	4402      	add	r2, r0
 80005aa:	4603      	mov	r3, r0
 80005ac:	4293      	cmp	r3, r2
 80005ae:	d100      	bne.n	80005b2 <memset+0xa>
 80005b0:	4770      	bx	lr
 80005b2:	f803 1b01 	strb.w	r1, [r3], #1
 80005b6:	e7f9      	b.n	80005ac <memset+0x4>

080005b8 <iprintf>:
 80005b8:	b40f      	push	{r0, r1, r2, r3}
 80005ba:	4b0a      	ldr	r3, [pc, #40]	; (80005e4 <iprintf+0x2c>)
 80005bc:	b513      	push	{r0, r1, r4, lr}
 80005be:	681c      	ldr	r4, [r3, #0]
 80005c0:	b124      	cbz	r4, 80005cc <iprintf+0x14>
 80005c2:	69a3      	ldr	r3, [r4, #24]
 80005c4:	b913      	cbnz	r3, 80005cc <iprintf+0x14>
 80005c6:	4620      	mov	r0, r4
 80005c8:	f000 f866 	bl	8000698 <__sinit>
 80005cc:	ab05      	add	r3, sp, #20
 80005ce:	9a04      	ldr	r2, [sp, #16]
 80005d0:	68a1      	ldr	r1, [r4, #8]
 80005d2:	9301      	str	r3, [sp, #4]
 80005d4:	4620      	mov	r0, r4
 80005d6:	f000 f983 	bl	80008e0 <_vfiprintf_r>
 80005da:	b002      	add	sp, #8
 80005dc:	e8bd 4010 	ldmia.w	sp!, {r4, lr}
 80005e0:	b004      	add	sp, #16
 80005e2:	4770      	bx	lr
 80005e4:	20000000 	.word	0x20000000

080005e8 <std>:
 80005e8:	2300      	movs	r3, #0
 80005ea:	b510      	push	{r4, lr}
 80005ec:	4604      	mov	r4, r0
 80005ee:	e9c0 3300 	strd	r3, r3, [r0]
 80005f2:	e9c0 3304 	strd	r3, r3, [r0, #16]
 80005f6:	6083      	str	r3, [r0, #8]
 80005f8:	8181      	strh	r1, [r0, #12]
 80005fa:	6643      	str	r3, [r0, #100]	; 0x64
 80005fc:	81c2      	strh	r2, [r0, #14]
 80005fe:	6183      	str	r3, [r0, #24]
 8000600:	4619      	mov	r1, r3
 8000602:	2208      	movs	r2, #8
 8000604:	305c      	adds	r0, #92	; 0x5c
 8000606:	f7ff ffcf 	bl	80005a8 <memset>
 800060a:	4b05      	ldr	r3, [pc, #20]	; (8000620 <std+0x38>)
 800060c:	6263      	str	r3, [r4, #36]	; 0x24
 800060e:	4b05      	ldr	r3, [pc, #20]	; (8000624 <std+0x3c>)
 8000610:	62a3      	str	r3, [r4, #40]	; 0x28
 8000612:	4b05      	ldr	r3, [pc, #20]	; (8000628 <std+0x40>)
 8000614:	62e3      	str	r3, [r4, #44]	; 0x2c
 8000616:	4b05      	ldr	r3, [pc, #20]	; (800062c <std+0x44>)
 8000618:	6224      	str	r4, [r4, #32]
 800061a:	6323      	str	r3, [r4, #48]	; 0x30
 800061c:	bd10      	pop	{r4, pc}
 800061e:	bf00      	nop
 8000620:	08000e89 	.word	0x08000e89
 8000624:	08000eab 	.word	0x08000eab
 8000628:	08000ee3 	.word	0x08000ee3
 800062c:	08000f07 	.word	0x08000f07

08000630 <_cleanup_r>:
 8000630:	4901      	ldr	r1, [pc, #4]	; (8000638 <_cleanup_r+0x8>)
 8000632:	f000 b8af 	b.w	8000794 <_fwalk_reent>
 8000636:	bf00      	nop
 8000638:	080011e1 	.word	0x080011e1

0800063c <__sfmoreglue>:
 800063c:	b570      	push	{r4, r5, r6, lr}
 800063e:	1e4a      	subs	r2, r1, #1
 8000640:	2568      	movs	r5, #104	; 0x68
 8000642:	4355      	muls	r5, r2
 8000644:	460e      	mov	r6, r1
 8000646:	f105 0174 	add.w	r1, r5, #116	; 0x74
 800064a:	f000 f8c5 	bl	80007d8 <_malloc_r>
 800064e:	4604      	mov	r4, r0
 8000650:	b140      	cbz	r0, 8000664 <__sfmoreglue+0x28>
 8000652:	2100      	movs	r1, #0
 8000654:	e9c0 1600 	strd	r1, r6, [r0]
 8000658:	300c      	adds	r0, #12
 800065a:	60a0      	str	r0, [r4, #8]
 800065c:	f105 0268 	add.w	r2, r5, #104	; 0x68
 8000660:	f7ff ffa2 	bl	80005a8 <memset>
 8000664:	4620      	mov	r0, r4
 8000666:	bd70      	pop	{r4, r5, r6, pc}

08000668 <__sfp_lock_acquire>:
 8000668:	4801      	ldr	r0, [pc, #4]	; (8000670 <__sfp_lock_acquire+0x8>)
 800066a:	f000 b8b3 	b.w	80007d4 <__retarget_lock_acquire_recursive>
 800066e:	bf00      	nop
 8000670:	20000094 	.word	0x20000094

08000674 <__sfp_lock_release>:
 8000674:	4801      	ldr	r0, [pc, #4]	; (800067c <__sfp_lock_release+0x8>)
 8000676:	f000 b8ae 	b.w	80007d6 <__retarget_lock_release_recursive>
 800067a:	bf00      	nop
 800067c:	20000094 	.word	0x20000094

08000680 <__sinit_lock_acquire>:
 8000680:	4801      	ldr	r0, [pc, #4]	; (8000688 <__sinit_lock_acquire+0x8>)
 8000682:	f000 b8a7 	b.w	80007d4 <__retarget_lock_acquire_recursive>
 8000686:	bf00      	nop
 8000688:	2000008f 	.word	0x2000008f

0800068c <__sinit_lock_release>:
 800068c:	4801      	ldr	r0, [pc, #4]	; (8000694 <__sinit_lock_release+0x8>)
 800068e:	f000 b8a2 	b.w	80007d6 <__retarget_lock_release_recursive>
 8000692:	bf00      	nop
 8000694:	2000008f 	.word	0x2000008f

08000698 <__sinit>:
 8000698:	b510      	push	{r4, lr}
 800069a:	4604      	mov	r4, r0
 800069c:	f7ff fff0 	bl	8000680 <__sinit_lock_acquire>
 80006a0:	69a3      	ldr	r3, [r4, #24]
 80006a2:	b11b      	cbz	r3, 80006ac <__sinit+0x14>
 80006a4:	e8bd 4010 	ldmia.w	sp!, {r4, lr}
 80006a8:	f7ff bff0 	b.w	800068c <__sinit_lock_release>
 80006ac:	e9c4 3312 	strd	r3, r3, [r4, #72]	; 0x48
 80006b0:	6523      	str	r3, [r4, #80]	; 0x50
 80006b2:	4b13      	ldr	r3, [pc, #76]	; (8000700 <__sinit+0x68>)
 80006b4:	4a13      	ldr	r2, [pc, #76]	; (8000704 <__sinit+0x6c>)
 80006b6:	681b      	ldr	r3, [r3, #0]
 80006b8:	62a2      	str	r2, [r4, #40]	; 0x28
 80006ba:	42a3      	cmp	r3, r4
 80006bc:	bf04      	itt	eq
 80006be:	2301      	moveq	r3, #1
 80006c0:	61a3      	streq	r3, [r4, #24]
 80006c2:	4620      	mov	r0, r4
 80006c4:	f000 f820 	bl	8000708 <__sfp>
 80006c8:	6060      	str	r0, [r4, #4]
 80006ca:	4620      	mov	r0, r4
 80006cc:	f000 f81c 	bl	8000708 <__sfp>
 80006d0:	60a0      	str	r0, [r4, #8]
 80006d2:	4620      	mov	r0, r4
 80006d4:	f000 f818 	bl	8000708 <__sfp>
 80006d8:	2200      	movs	r2, #0
 80006da:	60e0      	str	r0, [r4, #12]
 80006dc:	2104      	movs	r1, #4
 80006de:	6860      	ldr	r0, [r4, #4]
 80006e0:	f7ff ff82 	bl	80005e8 <std>
 80006e4:	68a0      	ldr	r0, [r4, #8]
 80006e6:	2201      	movs	r2, #1
 80006e8:	2109      	movs	r1, #9
 80006ea:	f7ff ff7d 	bl	80005e8 <std>
 80006ee:	68e0      	ldr	r0, [r4, #12]
 80006f0:	2202      	movs	r2, #2
 80006f2:	2112      	movs	r1, #18
 80006f4:	f7ff ff78 	bl	80005e8 <std>
 80006f8:	2301      	movs	r3, #1
 80006fa:	61a3      	str	r3, [r4, #24]
 80006fc:	e7d2      	b.n	80006a4 <__sinit+0xc>
 80006fe:	bf00      	nop
 8000700:	08001488 	.word	0x08001488
 8000704:	08000631 	.word	0x08000631

08000708 <__sfp>:
 8000708:	b5f8      	push	{r3, r4, r5, r6, r7, lr}
 800070a:	4607      	mov	r7, r0
 800070c:	f7ff ffac 	bl	8000668 <__sfp_lock_acquire>
 8000710:	4b1e      	ldr	r3, [pc, #120]	; (800078c <__sfp+0x84>)
 8000712:	681e      	ldr	r6, [r3, #0]
 8000714:	69b3      	ldr	r3, [r6, #24]
 8000716:	b913      	cbnz	r3, 800071e <__sfp+0x16>
 8000718:	4630      	mov	r0, r6
 800071a:	f7ff ffbd 	bl	8000698 <__sinit>
 800071e:	3648      	adds	r6, #72	; 0x48
 8000720:	e9d6 3401 	ldrd	r3, r4, [r6, #4]
 8000724:	3b01      	subs	r3, #1
 8000726:	d503      	bpl.n	8000730 <__sfp+0x28>
 8000728:	6833      	ldr	r3, [r6, #0]
 800072a:	b30b      	cbz	r3, 8000770 <__sfp+0x68>
 800072c:	6836      	ldr	r6, [r6, #0]
 800072e:	e7f7      	b.n	8000720 <__sfp+0x18>
 8000730:	f9b4 500c 	ldrsh.w	r5, [r4, #12]
 8000734:	b9d5      	cbnz	r5, 800076c <__sfp+0x64>
 8000736:	4b16      	ldr	r3, [pc, #88]	; (8000790 <__sfp+0x88>)
 8000738:	60e3      	str	r3, [r4, #12]
 800073a:	f104 0058 	add.w	r0, r4, #88	; 0x58
 800073e:	6665      	str	r5, [r4, #100]	; 0x64
 8000740:	f000 f847 	bl	80007d2 <__retarget_lock_init_recursive>
 8000744:	f7ff ff96 	bl	8000674 <__sfp_lock_release>
 8000748:	e9c4 5501 	strd	r5, r5, [r4, #4]
 800074c:	e9c4 5504 	strd	r5, r5, [r4, #16]
 8000750:	6025      	str	r5, [r4, #0]
 8000752:	61a5      	str	r5, [r4, #24]
 8000754:	2208      	movs	r2, #8
 8000756:	4629      	mov	r1, r5
 8000758:	f104 005c 	add.w	r0, r4, #92	; 0x5c
 800075c:	f7ff ff24 	bl	80005a8 <memset>
 8000760:	e9c4 550d 	strd	r5, r5, [r4, #52]	; 0x34
 8000764:	e9c4 5512 	strd	r5, r5, [r4, #72]	; 0x48
 8000768:	4620      	mov	r0, r4
 800076a:	bdf8      	pop	{r3, r4, r5, r6, r7, pc}
 800076c:	3468      	adds	r4, #104	; 0x68
 800076e:	e7d9      	b.n	8000724 <__sfp+0x1c>
 8000770:	2104      	movs	r1, #4
 8000772:	4638      	mov	r0, r7
 8000774:	f7ff ff62 	bl	800063c <__sfmoreglue>
 8000778:	4604      	mov	r4, r0
 800077a:	6030      	str	r0, [r6, #0]
 800077c:	2800      	cmp	r0, #0
 800077e:	d1d5      	bne.n	800072c <__sfp+0x24>
 8000780:	f7ff ff78 	bl	8000674 <__sfp_lock_release>
 8000784:	230c      	movs	r3, #12
 8000786:	603b      	str	r3, [r7, #0]
 8000788:	e7ee      	b.n	8000768 <__sfp+0x60>
 800078a:	bf00      	nop
 800078c:	08001488 	.word	0x08001488
 8000790:	ffff0001 	.word	0xffff0001

08000794 <_fwalk_reent>:
 8000794:	e92d 43f8 	stmdb	sp!, {r3, r4, r5, r6, r7, r8, r9, lr}
 8000798:	4606      	mov	r6, r0
 800079a:	4688      	mov	r8, r1
 800079c:	f100 0448 	add.w	r4, r0, #72	; 0x48
 80007a0:	2700      	movs	r7, #0
 80007a2:	e9d4 9501 	ldrd	r9, r5, [r4, #4]
 80007a6:	f1b9 0901 	subs.w	r9, r9, #1
 80007aa:	d505      	bpl.n	80007b8 <_fwalk_reent+0x24>
 80007ac:	6824      	ldr	r4, [r4, #0]
 80007ae:	2c00      	cmp	r4, #0
 80007b0:	d1f7      	bne.n	80007a2 <_fwalk_reent+0xe>
 80007b2:	4638      	mov	r0, r7
 80007b4:	e8bd 83f8 	ldmia.w	sp!, {r3, r4, r5, r6, r7, r8, r9, pc}
 80007b8:	89ab      	ldrh	r3, [r5, #12]
 80007ba:	2b01      	cmp	r3, #1
 80007bc:	d907      	bls.n	80007ce <_fwalk_reent+0x3a>
 80007be:	f9b5 300e 	ldrsh.w	r3, [r5, #14]
 80007c2:	3301      	adds	r3, #1
 80007c4:	d003      	beq.n	80007ce <_fwalk_reent+0x3a>
 80007c6:	4629      	mov	r1, r5
 80007c8:	4630      	mov	r0, r6
 80007ca:	47c0      	blx	r8
 80007cc:	4307      	orrs	r7, r0
 80007ce:	3568      	adds	r5, #104	; 0x68
 80007d0:	e7e9      	b.n	80007a6 <_fwalk_reent+0x12>

080007d2 <__retarget_lock_init_recursive>:
 80007d2:	4770      	bx	lr

080007d4 <__retarget_lock_acquire_recursive>:
 80007d4:	4770      	bx	lr

080007d6 <__retarget_lock_release_recursive>:
 80007d6:	4770      	bx	lr

080007d8 <_malloc_r>:
 80007d8:	b5f8      	push	{r3, r4, r5, r6, r7, lr}
 80007da:	1ccd      	adds	r5, r1, #3
 80007dc:	f025 0503 	bic.w	r5, r5, #3
 80007e0:	3508      	adds	r5, #8
 80007e2:	2d0c      	cmp	r5, #12
 80007e4:	bf38      	it	cc
 80007e6:	250c      	movcc	r5, #12
 80007e8:	2d00      	cmp	r5, #0
 80007ea:	4606      	mov	r6, r0
 80007ec:	db01      	blt.n	80007f2 <_malloc_r+0x1a>
 80007ee:	42a9      	cmp	r1, r5
 80007f0:	d903      	bls.n	80007fa <_malloc_r+0x22>
 80007f2:	230c      	movs	r3, #12
 80007f4:	6033      	str	r3, [r6, #0]
 80007f6:	2000      	movs	r0, #0
 80007f8:	bdf8      	pop	{r3, r4, r5, r6, r7, pc}
 80007fa:	f000 fda3 	bl	8001344 <__malloc_lock>
 80007fe:	4921      	ldr	r1, [pc, #132]	; (8000884 <_malloc_r+0xac>)
 8000800:	680a      	ldr	r2, [r1, #0]
 8000802:	4614      	mov	r4, r2
 8000804:	b99c      	cbnz	r4, 800082e <_malloc_r+0x56>
 8000806:	4f20      	ldr	r7, [pc, #128]	; (8000888 <_malloc_r+0xb0>)
 8000808:	683b      	ldr	r3, [r7, #0]
 800080a:	b923      	cbnz	r3, 8000816 <_malloc_r+0x3e>
 800080c:	4621      	mov	r1, r4
 800080e:	4630      	mov	r0, r6
 8000810:	f000 fb2a 	bl	8000e68 <_sbrk_r>
 8000814:	6038      	str	r0, [r7, #0]
 8000816:	4629      	mov	r1, r5
 8000818:	4630      	mov	r0, r6
 800081a:	f000 fb25 	bl	8000e68 <_sbrk_r>
 800081e:	1c43      	adds	r3, r0, #1
 8000820:	d123      	bne.n	800086a <_malloc_r+0x92>
 8000822:	230c      	movs	r3, #12
 8000824:	6033      	str	r3, [r6, #0]
 8000826:	4630      	mov	r0, r6
 8000828:	f000 fd92 	bl	8001350 <__malloc_unlock>
 800082c:	e7e3      	b.n	80007f6 <_malloc_r+0x1e>
 800082e:	6823      	ldr	r3, [r4, #0]
 8000830:	1b5b      	subs	r3, r3, r5
 8000832:	d417      	bmi.n	8000864 <_malloc_r+0x8c>
 8000834:	2b0b      	cmp	r3, #11
 8000836:	d903      	bls.n	8000840 <_malloc_r+0x68>
 8000838:	6023      	str	r3, [r4, #0]
 800083a:	441c      	add	r4, r3
 800083c:	6025      	str	r5, [r4, #0]
 800083e:	e004      	b.n	800084a <_malloc_r+0x72>
 8000840:	6863      	ldr	r3, [r4, #4]
 8000842:	42a2      	cmp	r2, r4
 8000844:	bf0c      	ite	eq
 8000846:	600b      	streq	r3, [r1, #0]
 8000848:	6053      	strne	r3, [r2, #4]
 800084a:	4630      	mov	r0, r6
 800084c:	f000 fd80 	bl	8001350 <__malloc_unlock>
 8000850:	f104 000b 	add.w	r0, r4, #11
 8000854:	1d23      	adds	r3, r4, #4
 8000856:	f020 0007 	bic.w	r0, r0, #7
 800085a:	1ac2      	subs	r2, r0, r3
 800085c:	d0cc      	beq.n	80007f8 <_malloc_r+0x20>
 800085e:	1a1b      	subs	r3, r3, r0
 8000860:	50a3      	str	r3, [r4, r2]
 8000862:	e7c9      	b.n	80007f8 <_malloc_r+0x20>
 8000864:	4622      	mov	r2, r4
 8000866:	6864      	ldr	r4, [r4, #4]
 8000868:	e7cc      	b.n	8000804 <_malloc_r+0x2c>
 800086a:	1cc4      	adds	r4, r0, #3
 800086c:	f024 0403 	bic.w	r4, r4, #3
 8000870:	42a0      	cmp	r0, r4
 8000872:	d0e3      	beq.n	800083c <_malloc_r+0x64>
 8000874:	1a21      	subs	r1, r4, r0
 8000876:	4630      	mov	r0, r6
 8000878:	f000 faf6 	bl	8000e68 <_sbrk_r>
 800087c:	3001      	adds	r0, #1
 800087e:	d1dd      	bne.n	800083c <_malloc_r+0x64>
 8000880:	e7cf      	b.n	8000822 <_malloc_r+0x4a>
 8000882:	bf00      	nop
 8000884:	20000084 	.word	0x20000084
 8000888:	20000088 	.word	0x20000088

0800088c <__sfputc_r>:
 800088c:	6893      	ldr	r3, [r2, #8]
 800088e:	3b01      	subs	r3, #1
 8000890:	2b00      	cmp	r3, #0
 8000892:	b410      	push	{r4}
 8000894:	6093      	str	r3, [r2, #8]
 8000896:	da08      	bge.n	80008aa <__sfputc_r+0x1e>
 8000898:	6994      	ldr	r4, [r2, #24]
 800089a:	42a3      	cmp	r3, r4
 800089c:	db01      	blt.n	80008a2 <__sfputc_r+0x16>
 800089e:	290a      	cmp	r1, #10
 80008a0:	d103      	bne.n	80008aa <__sfputc_r+0x1e>
 80008a2:	f85d 4b04 	ldr.w	r4, [sp], #4
 80008a6:	f000 bb33 	b.w	8000f10 <__swbuf_r>
 80008aa:	6813      	ldr	r3, [r2, #0]
 80008ac:	1c58      	adds	r0, r3, #1
 80008ae:	6010      	str	r0, [r2, #0]
 80008b0:	7019      	strb	r1, [r3, #0]
 80008b2:	4608      	mov	r0, r1
 80008b4:	f85d 4b04 	ldr.w	r4, [sp], #4
 80008b8:	4770      	bx	lr

080008ba <__sfputs_r>:
 80008ba:	b5f8      	push	{r3, r4, r5, r6, r7, lr}
 80008bc:	4606      	mov	r6, r0
 80008be:	460f      	mov	r7, r1
 80008c0:	4614      	mov	r4, r2
 80008c2:	18d5      	adds	r5, r2, r3
 80008c4:	42ac      	cmp	r4, r5
 80008c6:	d101      	bne.n	80008cc <__sfputs_r+0x12>
 80008c8:	2000      	movs	r0, #0
 80008ca:	e007      	b.n	80008dc <__sfputs_r+0x22>
 80008cc:	f814 1b01 	ldrb.w	r1, [r4], #1
 80008d0:	463a      	mov	r2, r7
 80008d2:	4630      	mov	r0, r6
 80008d4:	f7ff ffda 	bl	800088c <__sfputc_r>
 80008d8:	1c43      	adds	r3, r0, #1
 80008da:	d1f3      	bne.n	80008c4 <__sfputs_r+0xa>
 80008dc:	bdf8      	pop	{r3, r4, r5, r6, r7, pc}
	...

080008e0 <_vfiprintf_r>:
 80008e0:	e92d 4ff0 	stmdb	sp!, {r4, r5, r6, r7, r8, r9, sl, fp, lr}
 80008e4:	460d      	mov	r5, r1
 80008e6:	b09d      	sub	sp, #116	; 0x74
 80008e8:	4614      	mov	r4, r2
 80008ea:	4698      	mov	r8, r3
 80008ec:	4606      	mov	r6, r0
 80008ee:	b118      	cbz	r0, 80008f8 <_vfiprintf_r+0x18>
 80008f0:	6983      	ldr	r3, [r0, #24]
 80008f2:	b90b      	cbnz	r3, 80008f8 <_vfiprintf_r+0x18>
 80008f4:	f7ff fed0 	bl	8000698 <__sinit>
 80008f8:	4b89      	ldr	r3, [pc, #548]	; (8000b20 <_vfiprintf_r+0x240>)
 80008fa:	429d      	cmp	r5, r3
 80008fc:	d11b      	bne.n	8000936 <_vfiprintf_r+0x56>
 80008fe:	6875      	ldr	r5, [r6, #4]
 8000900:	6e6b      	ldr	r3, [r5, #100]	; 0x64
 8000902:	07d9      	lsls	r1, r3, #31
 8000904:	d405      	bmi.n	8000912 <_vfiprintf_r+0x32>
 8000906:	89ab      	ldrh	r3, [r5, #12]
 8000908:	059a      	lsls	r2, r3, #22
 800090a:	d402      	bmi.n	8000912 <_vfiprintf_r+0x32>
 800090c:	6da8      	ldr	r0, [r5, #88]	; 0x58
 800090e:	f7ff ff61 	bl	80007d4 <__retarget_lock_acquire_recursive>
 8000912:	89ab      	ldrh	r3, [r5, #12]
 8000914:	071b      	lsls	r3, r3, #28
 8000916:	d501      	bpl.n	800091c <_vfiprintf_r+0x3c>
 8000918:	692b      	ldr	r3, [r5, #16]
 800091a:	b9eb      	cbnz	r3, 8000958 <_vfiprintf_r+0x78>
 800091c:	4629      	mov	r1, r5
 800091e:	4630      	mov	r0, r6
 8000920:	f000 fb5a 	bl	8000fd8 <__swsetup_r>
 8000924:	b1c0      	cbz	r0, 8000958 <_vfiprintf_r+0x78>
 8000926:	6e6b      	ldr	r3, [r5, #100]	; 0x64
 8000928:	07dc      	lsls	r4, r3, #31
 800092a:	d50e      	bpl.n	800094a <_vfiprintf_r+0x6a>
 800092c:	f04f 30ff 	mov.w	r0, #4294967295
 8000930:	b01d      	add	sp, #116	; 0x74
 8000932:	e8bd 8ff0 	ldmia.w	sp!, {r4, r5, r6, r7, r8, r9, sl, fp, pc}
 8000936:	4b7b      	ldr	r3, [pc, #492]	; (8000b24 <_vfiprintf_r+0x244>)
 8000938:	429d      	cmp	r5, r3
 800093a:	d101      	bne.n	8000940 <_vfiprintf_r+0x60>
 800093c:	68b5      	ldr	r5, [r6, #8]
 800093e:	e7df      	b.n	8000900 <_vfiprintf_r+0x20>
 8000940:	4b79      	ldr	r3, [pc, #484]	; (8000b28 <_vfiprintf_r+0x248>)
 8000942:	429d      	cmp	r5, r3
 8000944:	bf08      	it	eq
 8000946:	68f5      	ldreq	r5, [r6, #12]
 8000948:	e7da      	b.n	8000900 <_vfiprintf_r+0x20>
 800094a:	89ab      	ldrh	r3, [r5, #12]
 800094c:	0598      	lsls	r0, r3, #22
 800094e:	d4ed      	bmi.n	800092c <_vfiprintf_r+0x4c>
 8000950:	6da8      	ldr	r0, [r5, #88]	; 0x58
 8000952:	f7ff ff40 	bl	80007d6 <__retarget_lock_release_recursive>
 8000956:	e7e9      	b.n	800092c <_vfiprintf_r+0x4c>
 8000958:	2300      	movs	r3, #0
 800095a:	9309      	str	r3, [sp, #36]	; 0x24
 800095c:	2320      	movs	r3, #32
 800095e:	f88d 3029 	strb.w	r3, [sp, #41]	; 0x29
 8000962:	f8cd 800c 	str.w	r8, [sp, #12]
 8000966:	2330      	movs	r3, #48	; 0x30
 8000968:	f8df 81c0 	ldr.w	r8, [pc, #448]	; 8000b2c <_vfiprintf_r+0x24c>
 800096c:	f88d 302a 	strb.w	r3, [sp, #42]	; 0x2a
 8000970:	f04f 0901 	mov.w	r9, #1
 8000974:	4623      	mov	r3, r4
 8000976:	469a      	mov	sl, r3
 8000978:	f813 2b01 	ldrb.w	r2, [r3], #1
 800097c:	b10a      	cbz	r2, 8000982 <_vfiprintf_r+0xa2>
 800097e:	2a25      	cmp	r2, #37	; 0x25
 8000980:	d1f9      	bne.n	8000976 <_vfiprintf_r+0x96>
 8000982:	ebba 0b04 	subs.w	fp, sl, r4
 8000986:	d00b      	beq.n	80009a0 <_vfiprintf_r+0xc0>
 8000988:	465b      	mov	r3, fp
 800098a:	4622      	mov	r2, r4
 800098c:	4629      	mov	r1, r5
 800098e:	4630      	mov	r0, r6
 8000990:	f7ff ff93 	bl	80008ba <__sfputs_r>
 8000994:	3001      	adds	r0, #1
 8000996:	f000 80aa 	beq.w	8000aee <_vfiprintf_r+0x20e>
 800099a:	9a09      	ldr	r2, [sp, #36]	; 0x24
 800099c:	445a      	add	r2, fp
 800099e:	9209      	str	r2, [sp, #36]	; 0x24
 80009a0:	f89a 3000 	ldrb.w	r3, [sl]
 80009a4:	2b00      	cmp	r3, #0
 80009a6:	f000 80a2 	beq.w	8000aee <_vfiprintf_r+0x20e>
 80009aa:	2300      	movs	r3, #0
 80009ac:	f04f 32ff 	mov.w	r2, #4294967295
 80009b0:	e9cd 2305 	strd	r2, r3, [sp, #20]
 80009b4:	f10a 0a01 	add.w	sl, sl, #1
 80009b8:	9304      	str	r3, [sp, #16]
 80009ba:	9307      	str	r3, [sp, #28]
 80009bc:	f88d 3053 	strb.w	r3, [sp, #83]	; 0x53
 80009c0:	931a      	str	r3, [sp, #104]	; 0x68
 80009c2:	4654      	mov	r4, sl
 80009c4:	2205      	movs	r2, #5
 80009c6:	f814 1b01 	ldrb.w	r1, [r4], #1
 80009ca:	4858      	ldr	r0, [pc, #352]	; (8000b2c <_vfiprintf_r+0x24c>)
 80009cc:	f7ff fc08 	bl	80001e0 <memchr>
 80009d0:	9a04      	ldr	r2, [sp, #16]
 80009d2:	b9d8      	cbnz	r0, 8000a0c <_vfiprintf_r+0x12c>
 80009d4:	06d1      	lsls	r1, r2, #27
 80009d6:	bf44      	itt	mi
 80009d8:	2320      	movmi	r3, #32
 80009da:	f88d 3053 	strbmi.w	r3, [sp, #83]	; 0x53
 80009de:	0713      	lsls	r3, r2, #28
 80009e0:	bf44      	itt	mi
 80009e2:	232b      	movmi	r3, #43	; 0x2b
 80009e4:	f88d 3053 	strbmi.w	r3, [sp, #83]	; 0x53
 80009e8:	f89a 3000 	ldrb.w	r3, [sl]
 80009ec:	2b2a      	cmp	r3, #42	; 0x2a
 80009ee:	d015      	beq.n	8000a1c <_vfiprintf_r+0x13c>
 80009f0:	9a07      	ldr	r2, [sp, #28]
 80009f2:	4654      	mov	r4, sl
 80009f4:	2000      	movs	r0, #0
 80009f6:	f04f 0c0a 	mov.w	ip, #10
 80009fa:	4621      	mov	r1, r4
 80009fc:	f811 3b01 	ldrb.w	r3, [r1], #1
 8000a00:	3b30      	subs	r3, #48	; 0x30
 8000a02:	2b09      	cmp	r3, #9
 8000a04:	d94e      	bls.n	8000aa4 <_vfiprintf_r+0x1c4>
 8000a06:	b1b0      	cbz	r0, 8000a36 <_vfiprintf_r+0x156>
 8000a08:	9207      	str	r2, [sp, #28]
 8000a0a:	e014      	b.n	8000a36 <_vfiprintf_r+0x156>
 8000a0c:	eba0 0308 	sub.w	r3, r0, r8
 8000a10:	fa09 f303 	lsl.w	r3, r9, r3
 8000a14:	4313      	orrs	r3, r2
 8000a16:	9304      	str	r3, [sp, #16]
 8000a18:	46a2      	mov	sl, r4
 8000a1a:	e7d2      	b.n	80009c2 <_vfiprintf_r+0xe2>
 8000a1c:	9b03      	ldr	r3, [sp, #12]
 8000a1e:	1d19      	adds	r1, r3, #4
 8000a20:	681b      	ldr	r3, [r3, #0]
 8000a22:	9103      	str	r1, [sp, #12]
 8000a24:	2b00      	cmp	r3, #0
 8000a26:	bfbb      	ittet	lt
 8000a28:	425b      	neglt	r3, r3
 8000a2a:	f042 0202 	orrlt.w	r2, r2, #2
 8000a2e:	9307      	strge	r3, [sp, #28]
 8000a30:	9307      	strlt	r3, [sp, #28]
 8000a32:	bfb8      	it	lt
 8000a34:	9204      	strlt	r2, [sp, #16]
 8000a36:	7823      	ldrb	r3, [r4, #0]
 8000a38:	2b2e      	cmp	r3, #46	; 0x2e
 8000a3a:	d10c      	bne.n	8000a56 <_vfiprintf_r+0x176>
 8000a3c:	7863      	ldrb	r3, [r4, #1]
 8000a3e:	2b2a      	cmp	r3, #42	; 0x2a
 8000a40:	d135      	bne.n	8000aae <_vfiprintf_r+0x1ce>
 8000a42:	9b03      	ldr	r3, [sp, #12]
 8000a44:	1d1a      	adds	r2, r3, #4
 8000a46:	681b      	ldr	r3, [r3, #0]
 8000a48:	9203      	str	r2, [sp, #12]
 8000a4a:	2b00      	cmp	r3, #0
 8000a4c:	bfb8      	it	lt
 8000a4e:	f04f 33ff 	movlt.w	r3, #4294967295
 8000a52:	3402      	adds	r4, #2
 8000a54:	9305      	str	r3, [sp, #20]
 8000a56:	f8df a0e4 	ldr.w	sl, [pc, #228]	; 8000b3c <_vfiprintf_r+0x25c>
 8000a5a:	7821      	ldrb	r1, [r4, #0]
 8000a5c:	2203      	movs	r2, #3
 8000a5e:	4650      	mov	r0, sl
 8000a60:	f7ff fbbe 	bl	80001e0 <memchr>
 8000a64:	b140      	cbz	r0, 8000a78 <_vfiprintf_r+0x198>
 8000a66:	2340      	movs	r3, #64	; 0x40
 8000a68:	eba0 000a 	sub.w	r0, r0, sl
 8000a6c:	fa03 f000 	lsl.w	r0, r3, r0
 8000a70:	9b04      	ldr	r3, [sp, #16]
 8000a72:	4303      	orrs	r3, r0
 8000a74:	3401      	adds	r4, #1
 8000a76:	9304      	str	r3, [sp, #16]
 8000a78:	f814 1b01 	ldrb.w	r1, [r4], #1
 8000a7c:	482c      	ldr	r0, [pc, #176]	; (8000b30 <_vfiprintf_r+0x250>)
 8000a7e:	f88d 1028 	strb.w	r1, [sp, #40]	; 0x28
 8000a82:	2206      	movs	r2, #6
 8000a84:	f7ff fbac 	bl	80001e0 <memchr>
 8000a88:	2800      	cmp	r0, #0
 8000a8a:	d03f      	beq.n	8000b0c <_vfiprintf_r+0x22c>
 8000a8c:	4b29      	ldr	r3, [pc, #164]	; (8000b34 <_vfiprintf_r+0x254>)
 8000a8e:	bb1b      	cbnz	r3, 8000ad8 <_vfiprintf_r+0x1f8>
 8000a90:	9b03      	ldr	r3, [sp, #12]
 8000a92:	3307      	adds	r3, #7
 8000a94:	f023 0307 	bic.w	r3, r3, #7
 8000a98:	3308      	adds	r3, #8
 8000a9a:	9303      	str	r3, [sp, #12]
 8000a9c:	9b09      	ldr	r3, [sp, #36]	; 0x24
 8000a9e:	443b      	add	r3, r7
 8000aa0:	9309      	str	r3, [sp, #36]	; 0x24
 8000aa2:	e767      	b.n	8000974 <_vfiprintf_r+0x94>
 8000aa4:	fb0c 3202 	mla	r2, ip, r2, r3
 8000aa8:	460c      	mov	r4, r1
 8000aaa:	2001      	movs	r0, #1
 8000aac:	e7a5      	b.n	80009fa <_vfiprintf_r+0x11a>
 8000aae:	2300      	movs	r3, #0
 8000ab0:	3401      	adds	r4, #1
 8000ab2:	9305      	str	r3, [sp, #20]
 8000ab4:	4619      	mov	r1, r3
 8000ab6:	f04f 0c0a 	mov.w	ip, #10
 8000aba:	4620      	mov	r0, r4
 8000abc:	f810 2b01 	ldrb.w	r2, [r0], #1
 8000ac0:	3a30      	subs	r2, #48	; 0x30
 8000ac2:	2a09      	cmp	r2, #9
 8000ac4:	d903      	bls.n	8000ace <_vfiprintf_r+0x1ee>
 8000ac6:	2b00      	cmp	r3, #0
 8000ac8:	d0c5      	beq.n	8000a56 <_vfiprintf_r+0x176>
 8000aca:	9105      	str	r1, [sp, #20]
 8000acc:	e7c3      	b.n	8000a56 <_vfiprintf_r+0x176>
 8000ace:	fb0c 2101 	mla	r1, ip, r1, r2
 8000ad2:	4604      	mov	r4, r0
 8000ad4:	2301      	movs	r3, #1
 8000ad6:	e7f0      	b.n	8000aba <_vfiprintf_r+0x1da>
 8000ad8:	ab03      	add	r3, sp, #12
 8000ada:	9300      	str	r3, [sp, #0]
 8000adc:	462a      	mov	r2, r5
 8000ade:	4b16      	ldr	r3, [pc, #88]	; (8000b38 <_vfiprintf_r+0x258>)
 8000ae0:	a904      	add	r1, sp, #16
 8000ae2:	4630      	mov	r0, r6
 8000ae4:	f3af 8000 	nop.w
 8000ae8:	4607      	mov	r7, r0
 8000aea:	1c78      	adds	r0, r7, #1
 8000aec:	d1d6      	bne.n	8000a9c <_vfiprintf_r+0x1bc>
 8000aee:	6e6b      	ldr	r3, [r5, #100]	; 0x64
 8000af0:	07d9      	lsls	r1, r3, #31
 8000af2:	d405      	bmi.n	8000b00 <_vfiprintf_r+0x220>
 8000af4:	89ab      	ldrh	r3, [r5, #12]
 8000af6:	059a      	lsls	r2, r3, #22
 8000af8:	d402      	bmi.n	8000b00 <_vfiprintf_r+0x220>
 8000afa:	6da8      	ldr	r0, [r5, #88]	; 0x58
 8000afc:	f7ff fe6b 	bl	80007d6 <__retarget_lock_release_recursive>
 8000b00:	89ab      	ldrh	r3, [r5, #12]
 8000b02:	065b      	lsls	r3, r3, #25
 8000b04:	f53f af12 	bmi.w	800092c <_vfiprintf_r+0x4c>
 8000b08:	9809      	ldr	r0, [sp, #36]	; 0x24
 8000b0a:	e711      	b.n	8000930 <_vfiprintf_r+0x50>
 8000b0c:	ab03      	add	r3, sp, #12
 8000b0e:	9300      	str	r3, [sp, #0]
 8000b10:	462a      	mov	r2, r5
 8000b12:	4b09      	ldr	r3, [pc, #36]	; (8000b38 <_vfiprintf_r+0x258>)
 8000b14:	a904      	add	r1, sp, #16
 8000b16:	4630      	mov	r0, r6
 8000b18:	f000 f880 	bl	8000c1c <_printf_i>
 8000b1c:	e7e4      	b.n	8000ae8 <_vfiprintf_r+0x208>
 8000b1e:	bf00      	nop
 8000b20:	080014ac 	.word	0x080014ac
 8000b24:	080014cc 	.word	0x080014cc
 8000b28:	0800148c 	.word	0x0800148c
 8000b2c:	080014ec 	.word	0x080014ec
 8000b30:	080014f6 	.word	0x080014f6
 8000b34:	00000000 	.word	0x00000000
 8000b38:	080008bb 	.word	0x080008bb
 8000b3c:	080014f2 	.word	0x080014f2

08000b40 <_printf_common>:
 8000b40:	e92d 47f0 	stmdb	sp!, {r4, r5, r6, r7, r8, r9, sl, lr}
 8000b44:	4616      	mov	r6, r2
 8000b46:	4699      	mov	r9, r3
 8000b48:	688a      	ldr	r2, [r1, #8]
 8000b4a:	690b      	ldr	r3, [r1, #16]
 8000b4c:	f8dd 8020 	ldr.w	r8, [sp, #32]
 8000b50:	4293      	cmp	r3, r2
 8000b52:	bfb8      	it	lt
 8000b54:	4613      	movlt	r3, r2
 8000b56:	6033      	str	r3, [r6, #0]
 8000b58:	f891 2043 	ldrb.w	r2, [r1, #67]	; 0x43
 8000b5c:	4607      	mov	r7, r0
 8000b5e:	460c      	mov	r4, r1
 8000b60:	b10a      	cbz	r2, 8000b66 <_printf_common+0x26>
 8000b62:	3301      	adds	r3, #1
 8000b64:	6033      	str	r3, [r6, #0]
 8000b66:	6823      	ldr	r3, [r4, #0]
 8000b68:	0699      	lsls	r1, r3, #26
 8000b6a:	bf42      	ittt	mi
 8000b6c:	6833      	ldrmi	r3, [r6, #0]
 8000b6e:	3302      	addmi	r3, #2
 8000b70:	6033      	strmi	r3, [r6, #0]
 8000b72:	6825      	ldr	r5, [r4, #0]
 8000b74:	f015 0506 	ands.w	r5, r5, #6
 8000b78:	d106      	bne.n	8000b88 <_printf_common+0x48>
 8000b7a:	f104 0a19 	add.w	sl, r4, #25
 8000b7e:	68e3      	ldr	r3, [r4, #12]
 8000b80:	6832      	ldr	r2, [r6, #0]
 8000b82:	1a9b      	subs	r3, r3, r2
 8000b84:	42ab      	cmp	r3, r5
 8000b86:	dc26      	bgt.n	8000bd6 <_printf_common+0x96>
 8000b88:	f894 2043 	ldrb.w	r2, [r4, #67]	; 0x43
 8000b8c:	1e13      	subs	r3, r2, #0
 8000b8e:	6822      	ldr	r2, [r4, #0]
 8000b90:	bf18      	it	ne
 8000b92:	2301      	movne	r3, #1
 8000b94:	0692      	lsls	r2, r2, #26
 8000b96:	d42b      	bmi.n	8000bf0 <_printf_common+0xb0>
 8000b98:	f104 0243 	add.w	r2, r4, #67	; 0x43
 8000b9c:	4649      	mov	r1, r9
 8000b9e:	4638      	mov	r0, r7
 8000ba0:	47c0      	blx	r8
 8000ba2:	3001      	adds	r0, #1
 8000ba4:	d01e      	beq.n	8000be4 <_printf_common+0xa4>
 8000ba6:	6823      	ldr	r3, [r4, #0]
 8000ba8:	68e5      	ldr	r5, [r4, #12]
 8000baa:	6832      	ldr	r2, [r6, #0]
 8000bac:	f003 0306 	and.w	r3, r3, #6
 8000bb0:	2b04      	cmp	r3, #4
 8000bb2:	bf08      	it	eq
 8000bb4:	1aad      	subeq	r5, r5, r2
 8000bb6:	68a3      	ldr	r3, [r4, #8]
 8000bb8:	6922      	ldr	r2, [r4, #16]
 8000bba:	bf0c      	ite	eq
 8000bbc:	ea25 75e5 	biceq.w	r5, r5, r5, asr #31
 8000bc0:	2500      	movne	r5, #0
 8000bc2:	4293      	cmp	r3, r2
 8000bc4:	bfc4      	itt	gt
 8000bc6:	1a9b      	subgt	r3, r3, r2
 8000bc8:	18ed      	addgt	r5, r5, r3
 8000bca:	2600      	movs	r6, #0
 8000bcc:	341a      	adds	r4, #26
 8000bce:	42b5      	cmp	r5, r6
 8000bd0:	d11a      	bne.n	8000c08 <_printf_common+0xc8>
 8000bd2:	2000      	movs	r0, #0
 8000bd4:	e008      	b.n	8000be8 <_printf_common+0xa8>
 8000bd6:	2301      	movs	r3, #1
 8000bd8:	4652      	mov	r2, sl
 8000bda:	4649      	mov	r1, r9
 8000bdc:	4638      	mov	r0, r7
 8000bde:	47c0      	blx	r8
 8000be0:	3001      	adds	r0, #1
 8000be2:	d103      	bne.n	8000bec <_printf_common+0xac>
 8000be4:	f04f 30ff 	mov.w	r0, #4294967295
 8000be8:	e8bd 87f0 	ldmia.w	sp!, {r4, r5, r6, r7, r8, r9, sl, pc}
 8000bec:	3501      	adds	r5, #1
 8000bee:	e7c6      	b.n	8000b7e <_printf_common+0x3e>
 8000bf0:	18e1      	adds	r1, r4, r3
 8000bf2:	1c5a      	adds	r2, r3, #1
 8000bf4:	2030      	movs	r0, #48	; 0x30
 8000bf6:	f881 0043 	strb.w	r0, [r1, #67]	; 0x43
 8000bfa:	4422      	add	r2, r4
 8000bfc:	f894 1045 	ldrb.w	r1, [r4, #69]	; 0x45
 8000c00:	f882 1043 	strb.w	r1, [r2, #67]	; 0x43
 8000c04:	3302      	adds	r3, #2
 8000c06:	e7c7      	b.n	8000b98 <_printf_common+0x58>
 8000c08:	2301      	movs	r3, #1
 8000c0a:	4622      	mov	r2, r4
 8000c0c:	4649      	mov	r1, r9
 8000c0e:	4638      	mov	r0, r7
 8000c10:	47c0      	blx	r8
 8000c12:	3001      	adds	r0, #1
 8000c14:	d0e6      	beq.n	8000be4 <_printf_common+0xa4>
 8000c16:	3601      	adds	r6, #1
 8000c18:	e7d9      	b.n	8000bce <_printf_common+0x8e>
	...

08000c1c <_printf_i>:
 8000c1c:	e92d 47ff 	stmdb	sp!, {r0, r1, r2, r3, r4, r5, r6, r7, r8, r9, sl, lr}
 8000c20:	460c      	mov	r4, r1
 8000c22:	4691      	mov	r9, r2
 8000c24:	7e27      	ldrb	r7, [r4, #24]
 8000c26:	990c      	ldr	r1, [sp, #48]	; 0x30
 8000c28:	2f78      	cmp	r7, #120	; 0x78
 8000c2a:	4680      	mov	r8, r0
 8000c2c:	469a      	mov	sl, r3
 8000c2e:	f104 0243 	add.w	r2, r4, #67	; 0x43
 8000c32:	d807      	bhi.n	8000c44 <_printf_i+0x28>
 8000c34:	2f62      	cmp	r7, #98	; 0x62
 8000c36:	d80a      	bhi.n	8000c4e <_printf_i+0x32>
 8000c38:	2f00      	cmp	r7, #0
 8000c3a:	f000 80d8 	beq.w	8000dee <_printf_i+0x1d2>
 8000c3e:	2f58      	cmp	r7, #88	; 0x58
 8000c40:	f000 80a3 	beq.w	8000d8a <_printf_i+0x16e>
 8000c44:	f104 0642 	add.w	r6, r4, #66	; 0x42
 8000c48:	f884 7042 	strb.w	r7, [r4, #66]	; 0x42
 8000c4c:	e03a      	b.n	8000cc4 <_printf_i+0xa8>
 8000c4e:	f1a7 0363 	sub.w	r3, r7, #99	; 0x63
 8000c52:	2b15      	cmp	r3, #21
 8000c54:	d8f6      	bhi.n	8000c44 <_printf_i+0x28>
 8000c56:	a001      	add	r0, pc, #4	; (adr r0, 8000c5c <_printf_i+0x40>)
 8000c58:	f850 f023 	ldr.w	pc, [r0, r3, lsl #2]
 8000c5c:	08000cb5 	.word	0x08000cb5
 8000c60:	08000cc9 	.word	0x08000cc9
 8000c64:	08000c45 	.word	0x08000c45
 8000c68:	08000c45 	.word	0x08000c45
 8000c6c:	08000c45 	.word	0x08000c45
 8000c70:	08000c45 	.word	0x08000c45
 8000c74:	08000cc9 	.word	0x08000cc9
 8000c78:	08000c45 	.word	0x08000c45
 8000c7c:	08000c45 	.word	0x08000c45
 8000c80:	08000c45 	.word	0x08000c45
 8000c84:	08000c45 	.word	0x08000c45
 8000c88:	08000dd5 	.word	0x08000dd5
 8000c8c:	08000cf9 	.word	0x08000cf9
 8000c90:	08000db7 	.word	0x08000db7
 8000c94:	08000c45 	.word	0x08000c45
 8000c98:	08000c45 	.word	0x08000c45
 8000c9c:	08000df7 	.word	0x08000df7
 8000ca0:	08000c45 	.word	0x08000c45
 8000ca4:	08000cf9 	.word	0x08000cf9
 8000ca8:	08000c45 	.word	0x08000c45
 8000cac:	08000c45 	.word	0x08000c45
 8000cb0:	08000dbf 	.word	0x08000dbf
 8000cb4:	680b      	ldr	r3, [r1, #0]
 8000cb6:	1d1a      	adds	r2, r3, #4
 8000cb8:	681b      	ldr	r3, [r3, #0]
 8000cba:	600a      	str	r2, [r1, #0]
 8000cbc:	f104 0642 	add.w	r6, r4, #66	; 0x42
 8000cc0:	f884 3042 	strb.w	r3, [r4, #66]	; 0x42
 8000cc4:	2301      	movs	r3, #1
 8000cc6:	e0a3      	b.n	8000e10 <_printf_i+0x1f4>
 8000cc8:	6825      	ldr	r5, [r4, #0]
 8000cca:	6808      	ldr	r0, [r1, #0]
 8000ccc:	062e      	lsls	r6, r5, #24
 8000cce:	f100 0304 	add.w	r3, r0, #4
 8000cd2:	d50a      	bpl.n	8000cea <_printf_i+0xce>
 8000cd4:	6805      	ldr	r5, [r0, #0]
 8000cd6:	600b      	str	r3, [r1, #0]
 8000cd8:	2d00      	cmp	r5, #0
 8000cda:	da03      	bge.n	8000ce4 <_printf_i+0xc8>
 8000cdc:	232d      	movs	r3, #45	; 0x2d
 8000cde:	426d      	negs	r5, r5
 8000ce0:	f884 3043 	strb.w	r3, [r4, #67]	; 0x43
 8000ce4:	485e      	ldr	r0, [pc, #376]	; (8000e60 <_printf_i+0x244>)
 8000ce6:	230a      	movs	r3, #10
 8000ce8:	e019      	b.n	8000d1e <_printf_i+0x102>
 8000cea:	f015 0f40 	tst.w	r5, #64	; 0x40
 8000cee:	6805      	ldr	r5, [r0, #0]
 8000cf0:	600b      	str	r3, [r1, #0]
 8000cf2:	bf18      	it	ne
 8000cf4:	b22d      	sxthne	r5, r5
 8000cf6:	e7ef      	b.n	8000cd8 <_printf_i+0xbc>
 8000cf8:	680b      	ldr	r3, [r1, #0]
 8000cfa:	6825      	ldr	r5, [r4, #0]
 8000cfc:	1d18      	adds	r0, r3, #4
 8000cfe:	6008      	str	r0, [r1, #0]
 8000d00:	0628      	lsls	r0, r5, #24
 8000d02:	d501      	bpl.n	8000d08 <_printf_i+0xec>
 8000d04:	681d      	ldr	r5, [r3, #0]
 8000d06:	e002      	b.n	8000d0e <_printf_i+0xf2>
 8000d08:	0669      	lsls	r1, r5, #25
 8000d0a:	d5fb      	bpl.n	8000d04 <_printf_i+0xe8>
 8000d0c:	881d      	ldrh	r5, [r3, #0]
 8000d0e:	4854      	ldr	r0, [pc, #336]	; (8000e60 <_printf_i+0x244>)
 8000d10:	2f6f      	cmp	r7, #111	; 0x6f
 8000d12:	bf0c      	ite	eq
 8000d14:	2308      	moveq	r3, #8
 8000d16:	230a      	movne	r3, #10
 8000d18:	2100      	movs	r1, #0
 8000d1a:	f884 1043 	strb.w	r1, [r4, #67]	; 0x43
 8000d1e:	6866      	ldr	r6, [r4, #4]
 8000d20:	60a6      	str	r6, [r4, #8]
 8000d22:	2e00      	cmp	r6, #0
 8000d24:	bfa2      	ittt	ge
 8000d26:	6821      	ldrge	r1, [r4, #0]
 8000d28:	f021 0104 	bicge.w	r1, r1, #4
 8000d2c:	6021      	strge	r1, [r4, #0]
 8000d2e:	b90d      	cbnz	r5, 8000d34 <_printf_i+0x118>
 8000d30:	2e00      	cmp	r6, #0
 8000d32:	d04d      	beq.n	8000dd0 <_printf_i+0x1b4>
 8000d34:	4616      	mov	r6, r2
 8000d36:	fbb5 f1f3 	udiv	r1, r5, r3
 8000d3a:	fb03 5711 	mls	r7, r3, r1, r5
 8000d3e:	5dc7      	ldrb	r7, [r0, r7]
 8000d40:	f806 7d01 	strb.w	r7, [r6, #-1]!
 8000d44:	462f      	mov	r7, r5
 8000d46:	42bb      	cmp	r3, r7
 8000d48:	460d      	mov	r5, r1
 8000d4a:	d9f4      	bls.n	8000d36 <_printf_i+0x11a>
 8000d4c:	2b08      	cmp	r3, #8
 8000d4e:	d10b      	bne.n	8000d68 <_printf_i+0x14c>
 8000d50:	6823      	ldr	r3, [r4, #0]
 8000d52:	07df      	lsls	r7, r3, #31
 8000d54:	d508      	bpl.n	8000d68 <_printf_i+0x14c>
 8000d56:	6923      	ldr	r3, [r4, #16]
 8000d58:	6861      	ldr	r1, [r4, #4]
 8000d5a:	4299      	cmp	r1, r3
 8000d5c:	bfde      	ittt	le
 8000d5e:	2330      	movle	r3, #48	; 0x30
 8000d60:	f806 3c01 	strble.w	r3, [r6, #-1]
 8000d64:	f106 36ff 	addle.w	r6, r6, #4294967295
 8000d68:	1b92      	subs	r2, r2, r6
 8000d6a:	6122      	str	r2, [r4, #16]
 8000d6c:	f8cd a000 	str.w	sl, [sp]
 8000d70:	464b      	mov	r3, r9
 8000d72:	aa03      	add	r2, sp, #12
 8000d74:	4621      	mov	r1, r4
 8000d76:	4640      	mov	r0, r8
 8000d78:	f7ff fee2 	bl	8000b40 <_printf_common>
 8000d7c:	3001      	adds	r0, #1
 8000d7e:	d14c      	bne.n	8000e1a <_printf_i+0x1fe>
 8000d80:	f04f 30ff 	mov.w	r0, #4294967295
 8000d84:	b004      	add	sp, #16
 8000d86:	e8bd 87f0 	ldmia.w	sp!, {r4, r5, r6, r7, r8, r9, sl, pc}
 8000d8a:	4835      	ldr	r0, [pc, #212]	; (8000e60 <_printf_i+0x244>)
 8000d8c:	f884 7045 	strb.w	r7, [r4, #69]	; 0x45
 8000d90:	6823      	ldr	r3, [r4, #0]
 8000d92:	680e      	ldr	r6, [r1, #0]
 8000d94:	061f      	lsls	r7, r3, #24
 8000d96:	f856 5b04 	ldr.w	r5, [r6], #4
 8000d9a:	600e      	str	r6, [r1, #0]
 8000d9c:	d514      	bpl.n	8000dc8 <_printf_i+0x1ac>
 8000d9e:	07d9      	lsls	r1, r3, #31
 8000da0:	bf44      	itt	mi
 8000da2:	f043 0320 	orrmi.w	r3, r3, #32
 8000da6:	6023      	strmi	r3, [r4, #0]
 8000da8:	b91d      	cbnz	r5, 8000db2 <_printf_i+0x196>
 8000daa:	6823      	ldr	r3, [r4, #0]
 8000dac:	f023 0320 	bic.w	r3, r3, #32
 8000db0:	6023      	str	r3, [r4, #0]
 8000db2:	2310      	movs	r3, #16
 8000db4:	e7b0      	b.n	8000d18 <_printf_i+0xfc>
 8000db6:	6823      	ldr	r3, [r4, #0]
 8000db8:	f043 0320 	orr.w	r3, r3, #32
 8000dbc:	6023      	str	r3, [r4, #0]
 8000dbe:	2378      	movs	r3, #120	; 0x78
 8000dc0:	4828      	ldr	r0, [pc, #160]	; (8000e64 <_printf_i+0x248>)
 8000dc2:	f884 3045 	strb.w	r3, [r4, #69]	; 0x45
 8000dc6:	e7e3      	b.n	8000d90 <_printf_i+0x174>
 8000dc8:	065e      	lsls	r6, r3, #25
 8000dca:	bf48      	it	mi
 8000dcc:	b2ad      	uxthmi	r5, r5
 8000dce:	e7e6      	b.n	8000d9e <_printf_i+0x182>
 8000dd0:	4616      	mov	r6, r2
 8000dd2:	e7bb      	b.n	8000d4c <_printf_i+0x130>
 8000dd4:	680b      	ldr	r3, [r1, #0]
 8000dd6:	6826      	ldr	r6, [r4, #0]
 8000dd8:	6960      	ldr	r0, [r4, #20]
 8000dda:	1d1d      	adds	r5, r3, #4
 8000ddc:	600d      	str	r5, [r1, #0]
 8000dde:	0635      	lsls	r5, r6, #24
 8000de0:	681b      	ldr	r3, [r3, #0]
 8000de2:	d501      	bpl.n	8000de8 <_printf_i+0x1cc>
 8000de4:	6018      	str	r0, [r3, #0]
 8000de6:	e002      	b.n	8000dee <_printf_i+0x1d2>
 8000de8:	0671      	lsls	r1, r6, #25
 8000dea:	d5fb      	bpl.n	8000de4 <_printf_i+0x1c8>
 8000dec:	8018      	strh	r0, [r3, #0]
 8000dee:	2300      	movs	r3, #0
 8000df0:	6123      	str	r3, [r4, #16]
 8000df2:	4616      	mov	r6, r2
 8000df4:	e7ba      	b.n	8000d6c <_printf_i+0x150>
 8000df6:	680b      	ldr	r3, [r1, #0]
 8000df8:	1d1a      	adds	r2, r3, #4
 8000dfa:	600a      	str	r2, [r1, #0]
 8000dfc:	681e      	ldr	r6, [r3, #0]
 8000dfe:	6862      	ldr	r2, [r4, #4]
 8000e00:	2100      	movs	r1, #0
 8000e02:	4630      	mov	r0, r6
 8000e04:	f7ff f9ec 	bl	80001e0 <memchr>
 8000e08:	b108      	cbz	r0, 8000e0e <_printf_i+0x1f2>
 8000e0a:	1b80      	subs	r0, r0, r6
 8000e0c:	6060      	str	r0, [r4, #4]
 8000e0e:	6863      	ldr	r3, [r4, #4]
 8000e10:	6123      	str	r3, [r4, #16]
 8000e12:	2300      	movs	r3, #0
 8000e14:	f884 3043 	strb.w	r3, [r4, #67]	; 0x43
 8000e18:	e7a8      	b.n	8000d6c <_printf_i+0x150>
 8000e1a:	6923      	ldr	r3, [r4, #16]
 8000e1c:	4632      	mov	r2, r6
 8000e1e:	4649      	mov	r1, r9
 8000e20:	4640      	mov	r0, r8
 8000e22:	47d0      	blx	sl
 8000e24:	3001      	adds	r0, #1
 8000e26:	d0ab      	beq.n	8000d80 <_printf_i+0x164>
 8000e28:	6823      	ldr	r3, [r4, #0]
 8000e2a:	079b      	lsls	r3, r3, #30
 8000e2c:	d413      	bmi.n	8000e56 <_printf_i+0x23a>
 8000e2e:	68e0      	ldr	r0, [r4, #12]
 8000e30:	9b03      	ldr	r3, [sp, #12]
 8000e32:	4298      	cmp	r0, r3
 8000e34:	bfb8      	it	lt
 8000e36:	4618      	movlt	r0, r3
 8000e38:	e7a4      	b.n	8000d84 <_printf_i+0x168>
 8000e3a:	2301      	movs	r3, #1
 8000e3c:	4632      	mov	r2, r6
 8000e3e:	4649      	mov	r1, r9
 8000e40:	4640      	mov	r0, r8
 8000e42:	47d0      	blx	sl
 8000e44:	3001      	adds	r0, #1
 8000e46:	d09b      	beq.n	8000d80 <_printf_i+0x164>
 8000e48:	3501      	adds	r5, #1
 8000e4a:	68e3      	ldr	r3, [r4, #12]
 8000e4c:	9903      	ldr	r1, [sp, #12]
 8000e4e:	1a5b      	subs	r3, r3, r1
 8000e50:	42ab      	cmp	r3, r5
 8000e52:	dcf2      	bgt.n	8000e3a <_printf_i+0x21e>
 8000e54:	e7eb      	b.n	8000e2e <_printf_i+0x212>
 8000e56:	2500      	movs	r5, #0
 8000e58:	f104 0619 	add.w	r6, r4, #25
 8000e5c:	e7f5      	b.n	8000e4a <_printf_i+0x22e>
 8000e5e:	bf00      	nop
 8000e60:	080014fd 	.word	0x080014fd
 8000e64:	0800150e 	.word	0x0800150e

08000e68 <_sbrk_r>:
 8000e68:	b538      	push	{r3, r4, r5, lr}
 8000e6a:	4d06      	ldr	r5, [pc, #24]	; (8000e84 <_sbrk_r+0x1c>)
 8000e6c:	2300      	movs	r3, #0
 8000e6e:	4604      	mov	r4, r0
 8000e70:	4608      	mov	r0, r1
 8000e72:	602b      	str	r3, [r5, #0]
 8000e74:	f7ff fb0e 	bl	8000494 <_sbrk>
 8000e78:	1c43      	adds	r3, r0, #1
 8000e7a:	d102      	bne.n	8000e82 <_sbrk_r+0x1a>
 8000e7c:	682b      	ldr	r3, [r5, #0]
 8000e7e:	b103      	cbz	r3, 8000e82 <_sbrk_r+0x1a>
 8000e80:	6023      	str	r3, [r4, #0]
 8000e82:	bd38      	pop	{r3, r4, r5, pc}
 8000e84:	20000098 	.word	0x20000098

08000e88 <__sread>:
 8000e88:	b510      	push	{r4, lr}
 8000e8a:	460c      	mov	r4, r1
 8000e8c:	f9b1 100e 	ldrsh.w	r1, [r1, #14]
 8000e90:	f000 fab4 	bl	80013fc <_read_r>
 8000e94:	2800      	cmp	r0, #0
 8000e96:	bfab      	itete	ge
 8000e98:	6d63      	ldrge	r3, [r4, #84]	; 0x54
 8000e9a:	89a3      	ldrhlt	r3, [r4, #12]
 8000e9c:	181b      	addge	r3, r3, r0
 8000e9e:	f423 5380 	biclt.w	r3, r3, #4096	; 0x1000
 8000ea2:	bfac      	ite	ge
 8000ea4:	6563      	strge	r3, [r4, #84]	; 0x54
 8000ea6:	81a3      	strhlt	r3, [r4, #12]
 8000ea8:	bd10      	pop	{r4, pc}

08000eaa <__swrite>:
 8000eaa:	e92d 41f0 	stmdb	sp!, {r4, r5, r6, r7, r8, lr}
 8000eae:	461f      	mov	r7, r3
 8000eb0:	898b      	ldrh	r3, [r1, #12]
 8000eb2:	05db      	lsls	r3, r3, #23
 8000eb4:	4605      	mov	r5, r0
 8000eb6:	460c      	mov	r4, r1
 8000eb8:	4616      	mov	r6, r2
 8000eba:	d505      	bpl.n	8000ec8 <__swrite+0x1e>
 8000ebc:	f9b1 100e 	ldrsh.w	r1, [r1, #14]
 8000ec0:	2302      	movs	r3, #2
 8000ec2:	2200      	movs	r2, #0
 8000ec4:	f000 f9c8 	bl	8001258 <_lseek_r>
 8000ec8:	89a3      	ldrh	r3, [r4, #12]
 8000eca:	f9b4 100e 	ldrsh.w	r1, [r4, #14]
 8000ece:	f423 5380 	bic.w	r3, r3, #4096	; 0x1000
 8000ed2:	81a3      	strh	r3, [r4, #12]
 8000ed4:	4632      	mov	r2, r6
 8000ed6:	463b      	mov	r3, r7
 8000ed8:	4628      	mov	r0, r5
 8000eda:	e8bd 41f0 	ldmia.w	sp!, {r4, r5, r6, r7, r8, lr}
 8000ede:	f000 b869 	b.w	8000fb4 <_write_r>

08000ee2 <__sseek>:
 8000ee2:	b510      	push	{r4, lr}
 8000ee4:	460c      	mov	r4, r1
 8000ee6:	f9b1 100e 	ldrsh.w	r1, [r1, #14]
 8000eea:	f000 f9b5 	bl	8001258 <_lseek_r>
 8000eee:	1c43      	adds	r3, r0, #1
 8000ef0:	89a3      	ldrh	r3, [r4, #12]
 8000ef2:	bf15      	itete	ne
 8000ef4:	6560      	strne	r0, [r4, #84]	; 0x54
 8000ef6:	f423 5380 	biceq.w	r3, r3, #4096	; 0x1000
 8000efa:	f443 5380 	orrne.w	r3, r3, #4096	; 0x1000
 8000efe:	81a3      	strheq	r3, [r4, #12]
 8000f00:	bf18      	it	ne
 8000f02:	81a3      	strhne	r3, [r4, #12]
 8000f04:	bd10      	pop	{r4, pc}

08000f06 <__sclose>:
 8000f06:	f9b1 100e 	ldrsh.w	r1, [r1, #14]
 8000f0a:	f000 b8d3 	b.w	80010b4 <_close_r>
	...

08000f10 <__swbuf_r>:
 8000f10:	b5f8      	push	{r3, r4, r5, r6, r7, lr}
 8000f12:	460e      	mov	r6, r1
 8000f14:	4614      	mov	r4, r2
 8000f16:	4605      	mov	r5, r0
 8000f18:	b118      	cbz	r0, 8000f22 <__swbuf_r+0x12>
 8000f1a:	6983      	ldr	r3, [r0, #24]
 8000f1c:	b90b      	cbnz	r3, 8000f22 <__swbuf_r+0x12>
 8000f1e:	f7ff fbbb 	bl	8000698 <__sinit>
 8000f22:	4b21      	ldr	r3, [pc, #132]	; (8000fa8 <__swbuf_r+0x98>)
 8000f24:	429c      	cmp	r4, r3
 8000f26:	d12b      	bne.n	8000f80 <__swbuf_r+0x70>
 8000f28:	686c      	ldr	r4, [r5, #4]
 8000f2a:	69a3      	ldr	r3, [r4, #24]
 8000f2c:	60a3      	str	r3, [r4, #8]
 8000f2e:	89a3      	ldrh	r3, [r4, #12]
 8000f30:	071a      	lsls	r2, r3, #28
 8000f32:	d52f      	bpl.n	8000f94 <__swbuf_r+0x84>
 8000f34:	6923      	ldr	r3, [r4, #16]
 8000f36:	b36b      	cbz	r3, 8000f94 <__swbuf_r+0x84>
 8000f38:	6923      	ldr	r3, [r4, #16]
 8000f3a:	6820      	ldr	r0, [r4, #0]
 8000f3c:	1ac0      	subs	r0, r0, r3
 8000f3e:	6963      	ldr	r3, [r4, #20]
 8000f40:	b2f6      	uxtb	r6, r6
 8000f42:	4283      	cmp	r3, r0
 8000f44:	4637      	mov	r7, r6
 8000f46:	dc04      	bgt.n	8000f52 <__swbuf_r+0x42>
 8000f48:	4621      	mov	r1, r4
 8000f4a:	4628      	mov	r0, r5
 8000f4c:	f000 f948 	bl	80011e0 <_fflush_r>
 8000f50:	bb30      	cbnz	r0, 8000fa0 <__swbuf_r+0x90>
 8000f52:	68a3      	ldr	r3, [r4, #8]
 8000f54:	3b01      	subs	r3, #1
 8000f56:	60a3      	str	r3, [r4, #8]
 8000f58:	6823      	ldr	r3, [r4, #0]
 8000f5a:	1c5a      	adds	r2, r3, #1
 8000f5c:	6022      	str	r2, [r4, #0]
 8000f5e:	701e      	strb	r6, [r3, #0]
 8000f60:	6963      	ldr	r3, [r4, #20]
 8000f62:	3001      	adds	r0, #1
 8000f64:	4283      	cmp	r3, r0
 8000f66:	d004      	beq.n	8000f72 <__swbuf_r+0x62>
 8000f68:	89a3      	ldrh	r3, [r4, #12]
 8000f6a:	07db      	lsls	r3, r3, #31
 8000f6c:	d506      	bpl.n	8000f7c <__swbuf_r+0x6c>
 8000f6e:	2e0a      	cmp	r6, #10
 8000f70:	d104      	bne.n	8000f7c <__swbuf_r+0x6c>
 8000f72:	4621      	mov	r1, r4
 8000f74:	4628      	mov	r0, r5
 8000f76:	f000 f933 	bl	80011e0 <_fflush_r>
 8000f7a:	b988      	cbnz	r0, 8000fa0 <__swbuf_r+0x90>
 8000f7c:	4638      	mov	r0, r7
 8000f7e:	bdf8      	pop	{r3, r4, r5, r6, r7, pc}
 8000f80:	4b0a      	ldr	r3, [pc, #40]	; (8000fac <__swbuf_r+0x9c>)
 8000f82:	429c      	cmp	r4, r3
 8000f84:	d101      	bne.n	8000f8a <__swbuf_r+0x7a>
 8000f86:	68ac      	ldr	r4, [r5, #8]
 8000f88:	e7cf      	b.n	8000f2a <__swbuf_r+0x1a>
 8000f8a:	4b09      	ldr	r3, [pc, #36]	; (8000fb0 <__swbuf_r+0xa0>)
 8000f8c:	429c      	cmp	r4, r3
 8000f8e:	bf08      	it	eq
 8000f90:	68ec      	ldreq	r4, [r5, #12]
 8000f92:	e7ca      	b.n	8000f2a <__swbuf_r+0x1a>
 8000f94:	4621      	mov	r1, r4
 8000f96:	4628      	mov	r0, r5
 8000f98:	f000 f81e 	bl	8000fd8 <__swsetup_r>
 8000f9c:	2800      	cmp	r0, #0
 8000f9e:	d0cb      	beq.n	8000f38 <__swbuf_r+0x28>
 8000fa0:	f04f 37ff 	mov.w	r7, #4294967295
 8000fa4:	e7ea      	b.n	8000f7c <__swbuf_r+0x6c>
 8000fa6:	bf00      	nop
 8000fa8:	080014ac 	.word	0x080014ac
 8000fac:	080014cc 	.word	0x080014cc
 8000fb0:	0800148c 	.word	0x0800148c

08000fb4 <_write_r>:
 8000fb4:	b538      	push	{r3, r4, r5, lr}
 8000fb6:	4d07      	ldr	r5, [pc, #28]	; (8000fd4 <_write_r+0x20>)
 8000fb8:	4604      	mov	r4, r0
 8000fba:	4608      	mov	r0, r1
 8000fbc:	4611      	mov	r1, r2
 8000fbe:	2200      	movs	r2, #0
 8000fc0:	602a      	str	r2, [r5, #0]
 8000fc2:	461a      	mov	r2, r3
 8000fc4:	f7ff fa16 	bl	80003f4 <_write>
 8000fc8:	1c43      	adds	r3, r0, #1
 8000fca:	d102      	bne.n	8000fd2 <_write_r+0x1e>
 8000fcc:	682b      	ldr	r3, [r5, #0]
 8000fce:	b103      	cbz	r3, 8000fd2 <_write_r+0x1e>
 8000fd0:	6023      	str	r3, [r4, #0]
 8000fd2:	bd38      	pop	{r3, r4, r5, pc}
 8000fd4:	20000098 	.word	0x20000098

08000fd8 <__swsetup_r>:
 8000fd8:	4b32      	ldr	r3, [pc, #200]	; (80010a4 <__swsetup_r+0xcc>)
 8000fda:	b570      	push	{r4, r5, r6, lr}
 8000fdc:	681d      	ldr	r5, [r3, #0]
 8000fde:	4606      	mov	r6, r0
 8000fe0:	460c      	mov	r4, r1
 8000fe2:	b125      	cbz	r5, 8000fee <__swsetup_r+0x16>
 8000fe4:	69ab      	ldr	r3, [r5, #24]
 8000fe6:	b913      	cbnz	r3, 8000fee <__swsetup_r+0x16>
 8000fe8:	4628      	mov	r0, r5
 8000fea:	f7ff fb55 	bl	8000698 <__sinit>
 8000fee:	4b2e      	ldr	r3, [pc, #184]	; (80010a8 <__swsetup_r+0xd0>)
 8000ff0:	429c      	cmp	r4, r3
 8000ff2:	d10f      	bne.n	8001014 <__swsetup_r+0x3c>
 8000ff4:	686c      	ldr	r4, [r5, #4]
 8000ff6:	89a3      	ldrh	r3, [r4, #12]
 8000ff8:	f9b4 200c 	ldrsh.w	r2, [r4, #12]
 8000ffc:	0719      	lsls	r1, r3, #28
 8000ffe:	d42c      	bmi.n	800105a <__swsetup_r+0x82>
 8001000:	06dd      	lsls	r5, r3, #27
 8001002:	d411      	bmi.n	8001028 <__swsetup_r+0x50>
 8001004:	2309      	movs	r3, #9
 8001006:	6033      	str	r3, [r6, #0]
 8001008:	f042 0340 	orr.w	r3, r2, #64	; 0x40
 800100c:	81a3      	strh	r3, [r4, #12]
 800100e:	f04f 30ff 	mov.w	r0, #4294967295
 8001012:	e03e      	b.n	8001092 <__swsetup_r+0xba>
 8001014:	4b25      	ldr	r3, [pc, #148]	; (80010ac <__swsetup_r+0xd4>)
 8001016:	429c      	cmp	r4, r3
 8001018:	d101      	bne.n	800101e <__swsetup_r+0x46>
 800101a:	68ac      	ldr	r4, [r5, #8]
 800101c:	e7eb      	b.n	8000ff6 <__swsetup_r+0x1e>
 800101e:	4b24      	ldr	r3, [pc, #144]	; (80010b0 <__swsetup_r+0xd8>)
 8001020:	429c      	cmp	r4, r3
 8001022:	bf08      	it	eq
 8001024:	68ec      	ldreq	r4, [r5, #12]
 8001026:	e7e6      	b.n	8000ff6 <__swsetup_r+0x1e>
 8001028:	0758      	lsls	r0, r3, #29
 800102a:	d512      	bpl.n	8001052 <__swsetup_r+0x7a>
 800102c:	6b61      	ldr	r1, [r4, #52]	; 0x34
 800102e:	b141      	cbz	r1, 8001042 <__swsetup_r+0x6a>
 8001030:	f104 0344 	add.w	r3, r4, #68	; 0x44
 8001034:	4299      	cmp	r1, r3
 8001036:	d002      	beq.n	800103e <__swsetup_r+0x66>
 8001038:	4630      	mov	r0, r6
 800103a:	f000 f98f 	bl	800135c <_free_r>
 800103e:	2300      	movs	r3, #0
 8001040:	6363      	str	r3, [r4, #52]	; 0x34
 8001042:	89a3      	ldrh	r3, [r4, #12]
 8001044:	f023 0324 	bic.w	r3, r3, #36	; 0x24
 8001048:	81a3      	strh	r3, [r4, #12]
 800104a:	2300      	movs	r3, #0
 800104c:	6063      	str	r3, [r4, #4]
 800104e:	6923      	ldr	r3, [r4, #16]
 8001050:	6023      	str	r3, [r4, #0]
 8001052:	89a3      	ldrh	r3, [r4, #12]
 8001054:	f043 0308 	orr.w	r3, r3, #8
 8001058:	81a3      	strh	r3, [r4, #12]
 800105a:	6923      	ldr	r3, [r4, #16]
 800105c:	b94b      	cbnz	r3, 8001072 <__swsetup_r+0x9a>
 800105e:	89a3      	ldrh	r3, [r4, #12]
 8001060:	f403 7320 	and.w	r3, r3, #640	; 0x280
 8001064:	f5b3 7f00 	cmp.w	r3, #512	; 0x200
 8001068:	d003      	beq.n	8001072 <__swsetup_r+0x9a>
 800106a:	4621      	mov	r1, r4
 800106c:	4630      	mov	r0, r6
 800106e:	f000 f929 	bl	80012c4 <__smakebuf_r>
 8001072:	89a0      	ldrh	r0, [r4, #12]
 8001074:	f9b4 200c 	ldrsh.w	r2, [r4, #12]
 8001078:	f010 0301 	ands.w	r3, r0, #1
 800107c:	d00a      	beq.n	8001094 <__swsetup_r+0xbc>
 800107e:	2300      	movs	r3, #0
 8001080:	60a3      	str	r3, [r4, #8]
 8001082:	6963      	ldr	r3, [r4, #20]
 8001084:	425b      	negs	r3, r3
 8001086:	61a3      	str	r3, [r4, #24]
 8001088:	6923      	ldr	r3, [r4, #16]
 800108a:	b943      	cbnz	r3, 800109e <__swsetup_r+0xc6>
 800108c:	f010 0080 	ands.w	r0, r0, #128	; 0x80
 8001090:	d1ba      	bne.n	8001008 <__swsetup_r+0x30>
 8001092:	bd70      	pop	{r4, r5, r6, pc}
 8001094:	0781      	lsls	r1, r0, #30
 8001096:	bf58      	it	pl
 8001098:	6963      	ldrpl	r3, [r4, #20]
 800109a:	60a3      	str	r3, [r4, #8]
 800109c:	e7f4      	b.n	8001088 <__swsetup_r+0xb0>
 800109e:	2000      	movs	r0, #0
 80010a0:	e7f7      	b.n	8001092 <__swsetup_r+0xba>
 80010a2:	bf00      	nop
 80010a4:	20000000 	.word	0x20000000
 80010a8:	080014ac 	.word	0x080014ac
 80010ac:	080014cc 	.word	0x080014cc
 80010b0:	0800148c 	.word	0x0800148c

080010b4 <_close_r>:
 80010b4:	b538      	push	{r3, r4, r5, lr}
 80010b6:	4d06      	ldr	r5, [pc, #24]	; (80010d0 <_close_r+0x1c>)
 80010b8:	2300      	movs	r3, #0
 80010ba:	4604      	mov	r4, r0
 80010bc:	4608      	mov	r0, r1
 80010be:	602b      	str	r3, [r5, #0]
 80010c0:	f7ff f9b4 	bl	800042c <_close>
 80010c4:	1c43      	adds	r3, r0, #1
 80010c6:	d102      	bne.n	80010ce <_close_r+0x1a>
 80010c8:	682b      	ldr	r3, [r5, #0]
 80010ca:	b103      	cbz	r3, 80010ce <_close_r+0x1a>
 80010cc:	6023      	str	r3, [r4, #0]
 80010ce:	bd38      	pop	{r3, r4, r5, pc}
 80010d0:	20000098 	.word	0x20000098

080010d4 <__sflush_r>:
 80010d4:	898a      	ldrh	r2, [r1, #12]
 80010d6:	e92d 41f0 	stmdb	sp!, {r4, r5, r6, r7, r8, lr}
 80010da:	4605      	mov	r5, r0
 80010dc:	0710      	lsls	r0, r2, #28
 80010de:	460c      	mov	r4, r1
 80010e0:	d458      	bmi.n	8001194 <__sflush_r+0xc0>
 80010e2:	684b      	ldr	r3, [r1, #4]
 80010e4:	2b00      	cmp	r3, #0
 80010e6:	dc05      	bgt.n	80010f4 <__sflush_r+0x20>
 80010e8:	6c0b      	ldr	r3, [r1, #64]	; 0x40
 80010ea:	2b00      	cmp	r3, #0
 80010ec:	dc02      	bgt.n	80010f4 <__sflush_r+0x20>
 80010ee:	2000      	movs	r0, #0
 80010f0:	e8bd 81f0 	ldmia.w	sp!, {r4, r5, r6, r7, r8, pc}
 80010f4:	6ae6      	ldr	r6, [r4, #44]	; 0x2c
 80010f6:	2e00      	cmp	r6, #0
 80010f8:	d0f9      	beq.n	80010ee <__sflush_r+0x1a>
 80010fa:	2300      	movs	r3, #0
 80010fc:	f412 5280 	ands.w	r2, r2, #4096	; 0x1000
 8001100:	682f      	ldr	r7, [r5, #0]
 8001102:	602b      	str	r3, [r5, #0]
 8001104:	d032      	beq.n	800116c <__sflush_r+0x98>
 8001106:	6d60      	ldr	r0, [r4, #84]	; 0x54
 8001108:	89a3      	ldrh	r3, [r4, #12]
 800110a:	075a      	lsls	r2, r3, #29
 800110c:	d505      	bpl.n	800111a <__sflush_r+0x46>
 800110e:	6863      	ldr	r3, [r4, #4]
 8001110:	1ac0      	subs	r0, r0, r3
 8001112:	6b63      	ldr	r3, [r4, #52]	; 0x34
 8001114:	b10b      	cbz	r3, 800111a <__sflush_r+0x46>
 8001116:	6c23      	ldr	r3, [r4, #64]	; 0x40
 8001118:	1ac0      	subs	r0, r0, r3
 800111a:	2300      	movs	r3, #0
 800111c:	4602      	mov	r2, r0
 800111e:	6ae6      	ldr	r6, [r4, #44]	; 0x2c
 8001120:	6a21      	ldr	r1, [r4, #32]
 8001122:	4628      	mov	r0, r5
 8001124:	47b0      	blx	r6
 8001126:	1c43      	adds	r3, r0, #1
 8001128:	89a3      	ldrh	r3, [r4, #12]
 800112a:	d106      	bne.n	800113a <__sflush_r+0x66>
 800112c:	6829      	ldr	r1, [r5, #0]
 800112e:	291d      	cmp	r1, #29
 8001130:	d82c      	bhi.n	800118c <__sflush_r+0xb8>
 8001132:	4a2a      	ldr	r2, [pc, #168]	; (80011dc <__sflush_r+0x108>)
 8001134:	40ca      	lsrs	r2, r1
 8001136:	07d6      	lsls	r6, r2, #31
 8001138:	d528      	bpl.n	800118c <__sflush_r+0xb8>
 800113a:	2200      	movs	r2, #0
 800113c:	6062      	str	r2, [r4, #4]
 800113e:	04d9      	lsls	r1, r3, #19
 8001140:	6922      	ldr	r2, [r4, #16]
 8001142:	6022      	str	r2, [r4, #0]
 8001144:	d504      	bpl.n	8001150 <__sflush_r+0x7c>
 8001146:	1c42      	adds	r2, r0, #1
 8001148:	d101      	bne.n	800114e <__sflush_r+0x7a>
 800114a:	682b      	ldr	r3, [r5, #0]
 800114c:	b903      	cbnz	r3, 8001150 <__sflush_r+0x7c>
 800114e:	6560      	str	r0, [r4, #84]	; 0x54
 8001150:	6b61      	ldr	r1, [r4, #52]	; 0x34
 8001152:	602f      	str	r7, [r5, #0]
 8001154:	2900      	cmp	r1, #0
 8001156:	d0ca      	beq.n	80010ee <__sflush_r+0x1a>
 8001158:	f104 0344 	add.w	r3, r4, #68	; 0x44
 800115c:	4299      	cmp	r1, r3
 800115e:	d002      	beq.n	8001166 <__sflush_r+0x92>
 8001160:	4628      	mov	r0, r5
 8001162:	f000 f8fb 	bl	800135c <_free_r>
 8001166:	2000      	movs	r0, #0
 8001168:	6360      	str	r0, [r4, #52]	; 0x34
 800116a:	e7c1      	b.n	80010f0 <__sflush_r+0x1c>
 800116c:	6a21      	ldr	r1, [r4, #32]
 800116e:	2301      	movs	r3, #1
 8001170:	4628      	mov	r0, r5
 8001172:	47b0      	blx	r6
 8001174:	1c41      	adds	r1, r0, #1
 8001176:	d1c7      	bne.n	8001108 <__sflush_r+0x34>
 8001178:	682b      	ldr	r3, [r5, #0]
 800117a:	2b00      	cmp	r3, #0
 800117c:	d0c4      	beq.n	8001108 <__sflush_r+0x34>
 800117e:	2b1d      	cmp	r3, #29
 8001180:	d001      	beq.n	8001186 <__sflush_r+0xb2>
 8001182:	2b16      	cmp	r3, #22
 8001184:	d101      	bne.n	800118a <__sflush_r+0xb6>
 8001186:	602f      	str	r7, [r5, #0]
 8001188:	e7b1      	b.n	80010ee <__sflush_r+0x1a>
 800118a:	89a3      	ldrh	r3, [r4, #12]
 800118c:	f043 0340 	orr.w	r3, r3, #64	; 0x40
 8001190:	81a3      	strh	r3, [r4, #12]
 8001192:	e7ad      	b.n	80010f0 <__sflush_r+0x1c>
 8001194:	690f      	ldr	r7, [r1, #16]
 8001196:	2f00      	cmp	r7, #0
 8001198:	d0a9      	beq.n	80010ee <__sflush_r+0x1a>
 800119a:	0793      	lsls	r3, r2, #30
 800119c:	680e      	ldr	r6, [r1, #0]
 800119e:	bf08      	it	eq
 80011a0:	694b      	ldreq	r3, [r1, #20]
 80011a2:	600f      	str	r7, [r1, #0]
 80011a4:	bf18      	it	ne
 80011a6:	2300      	movne	r3, #0
 80011a8:	eba6 0807 	sub.w	r8, r6, r7
 80011ac:	608b      	str	r3, [r1, #8]
 80011ae:	f1b8 0f00 	cmp.w	r8, #0
 80011b2:	dd9c      	ble.n	80010ee <__sflush_r+0x1a>
 80011b4:	6a21      	ldr	r1, [r4, #32]
 80011b6:	6aa6      	ldr	r6, [r4, #40]	; 0x28
 80011b8:	4643      	mov	r3, r8
 80011ba:	463a      	mov	r2, r7
 80011bc:	4628      	mov	r0, r5
 80011be:	47b0      	blx	r6
 80011c0:	2800      	cmp	r0, #0
 80011c2:	dc06      	bgt.n	80011d2 <__sflush_r+0xfe>
 80011c4:	89a3      	ldrh	r3, [r4, #12]
 80011c6:	f043 0340 	orr.w	r3, r3, #64	; 0x40
 80011ca:	81a3      	strh	r3, [r4, #12]
 80011cc:	f04f 30ff 	mov.w	r0, #4294967295
 80011d0:	e78e      	b.n	80010f0 <__sflush_r+0x1c>
 80011d2:	4407      	add	r7, r0
 80011d4:	eba8 0800 	sub.w	r8, r8, r0
 80011d8:	e7e9      	b.n	80011ae <__sflush_r+0xda>
 80011da:	bf00      	nop
 80011dc:	20400001 	.word	0x20400001

080011e0 <_fflush_r>:
 80011e0:	b538      	push	{r3, r4, r5, lr}
 80011e2:	690b      	ldr	r3, [r1, #16]
 80011e4:	4605      	mov	r5, r0
 80011e6:	460c      	mov	r4, r1
 80011e8:	b913      	cbnz	r3, 80011f0 <_fflush_r+0x10>
 80011ea:	2500      	movs	r5, #0
 80011ec:	4628      	mov	r0, r5
 80011ee:	bd38      	pop	{r3, r4, r5, pc}
 80011f0:	b118      	cbz	r0, 80011fa <_fflush_r+0x1a>
 80011f2:	6983      	ldr	r3, [r0, #24]
 80011f4:	b90b      	cbnz	r3, 80011fa <_fflush_r+0x1a>
 80011f6:	f7ff fa4f 	bl	8000698 <__sinit>
 80011fa:	4b14      	ldr	r3, [pc, #80]	; (800124c <_fflush_r+0x6c>)
 80011fc:	429c      	cmp	r4, r3
 80011fe:	d11b      	bne.n	8001238 <_fflush_r+0x58>
 8001200:	686c      	ldr	r4, [r5, #4]
 8001202:	f9b4 300c 	ldrsh.w	r3, [r4, #12]
 8001206:	2b00      	cmp	r3, #0
 8001208:	d0ef      	beq.n	80011ea <_fflush_r+0xa>
 800120a:	6e62      	ldr	r2, [r4, #100]	; 0x64
 800120c:	07d0      	lsls	r0, r2, #31
 800120e:	d404      	bmi.n	800121a <_fflush_r+0x3a>
 8001210:	0599      	lsls	r1, r3, #22
 8001212:	d402      	bmi.n	800121a <_fflush_r+0x3a>
 8001214:	6da0      	ldr	r0, [r4, #88]	; 0x58
 8001216:	f7ff fadd 	bl	80007d4 <__retarget_lock_acquire_recursive>
 800121a:	4628      	mov	r0, r5
 800121c:	4621      	mov	r1, r4
 800121e:	f7ff ff59 	bl	80010d4 <__sflush_r>
 8001222:	6e63      	ldr	r3, [r4, #100]	; 0x64
 8001224:	07da      	lsls	r2, r3, #31
 8001226:	4605      	mov	r5, r0
 8001228:	d4e0      	bmi.n	80011ec <_fflush_r+0xc>
 800122a:	89a3      	ldrh	r3, [r4, #12]
 800122c:	059b      	lsls	r3, r3, #22
 800122e:	d4dd      	bmi.n	80011ec <_fflush_r+0xc>
 8001230:	6da0      	ldr	r0, [r4, #88]	; 0x58
 8001232:	f7ff fad0 	bl	80007d6 <__retarget_lock_release_recursive>
 8001236:	e7d9      	b.n	80011ec <_fflush_r+0xc>
 8001238:	4b05      	ldr	r3, [pc, #20]	; (8001250 <_fflush_r+0x70>)
 800123a:	429c      	cmp	r4, r3
 800123c:	d101      	bne.n	8001242 <_fflush_r+0x62>
 800123e:	68ac      	ldr	r4, [r5, #8]
 8001240:	e7df      	b.n	8001202 <_fflush_r+0x22>
 8001242:	4b04      	ldr	r3, [pc, #16]	; (8001254 <_fflush_r+0x74>)
 8001244:	429c      	cmp	r4, r3
 8001246:	bf08      	it	eq
 8001248:	68ec      	ldreq	r4, [r5, #12]
 800124a:	e7da      	b.n	8001202 <_fflush_r+0x22>
 800124c:	080014ac 	.word	0x080014ac
 8001250:	080014cc 	.word	0x080014cc
 8001254:	0800148c 	.word	0x0800148c

08001258 <_lseek_r>:
 8001258:	b538      	push	{r3, r4, r5, lr}
 800125a:	4d07      	ldr	r5, [pc, #28]	; (8001278 <_lseek_r+0x20>)
 800125c:	4604      	mov	r4, r0
 800125e:	4608      	mov	r0, r1
 8001260:	4611      	mov	r1, r2
 8001262:	2200      	movs	r2, #0
 8001264:	602a      	str	r2, [r5, #0]
 8001266:	461a      	mov	r2, r3
 8001268:	f7ff f907 	bl	800047a <_lseek>
 800126c:	1c43      	adds	r3, r0, #1
 800126e:	d102      	bne.n	8001276 <_lseek_r+0x1e>
 8001270:	682b      	ldr	r3, [r5, #0]
 8001272:	b103      	cbz	r3, 8001276 <_lseek_r+0x1e>
 8001274:	6023      	str	r3, [r4, #0]
 8001276:	bd38      	pop	{r3, r4, r5, pc}
 8001278:	20000098 	.word	0x20000098

0800127c <__swhatbuf_r>:
 800127c:	b570      	push	{r4, r5, r6, lr}
 800127e:	460e      	mov	r6, r1
 8001280:	f9b1 100e 	ldrsh.w	r1, [r1, #14]
 8001284:	2900      	cmp	r1, #0
 8001286:	b096      	sub	sp, #88	; 0x58
 8001288:	4614      	mov	r4, r2
 800128a:	461d      	mov	r5, r3
 800128c:	da07      	bge.n	800129e <__swhatbuf_r+0x22>
 800128e:	2300      	movs	r3, #0
 8001290:	602b      	str	r3, [r5, #0]
 8001292:	89b3      	ldrh	r3, [r6, #12]
 8001294:	061a      	lsls	r2, r3, #24
 8001296:	d410      	bmi.n	80012ba <__swhatbuf_r+0x3e>
 8001298:	f44f 6380 	mov.w	r3, #1024	; 0x400
 800129c:	e00e      	b.n	80012bc <__swhatbuf_r+0x40>
 800129e:	466a      	mov	r2, sp
 80012a0:	f000 f8be 	bl	8001420 <_fstat_r>
 80012a4:	2800      	cmp	r0, #0
 80012a6:	dbf2      	blt.n	800128e <__swhatbuf_r+0x12>
 80012a8:	9a01      	ldr	r2, [sp, #4]
 80012aa:	f402 4270 	and.w	r2, r2, #61440	; 0xf000
 80012ae:	f5a2 5300 	sub.w	r3, r2, #8192	; 0x2000
 80012b2:	425a      	negs	r2, r3
 80012b4:	415a      	adcs	r2, r3
 80012b6:	602a      	str	r2, [r5, #0]
 80012b8:	e7ee      	b.n	8001298 <__swhatbuf_r+0x1c>
 80012ba:	2340      	movs	r3, #64	; 0x40
 80012bc:	2000      	movs	r0, #0
 80012be:	6023      	str	r3, [r4, #0]
 80012c0:	b016      	add	sp, #88	; 0x58
 80012c2:	bd70      	pop	{r4, r5, r6, pc}

080012c4 <__smakebuf_r>:
 80012c4:	898b      	ldrh	r3, [r1, #12]
 80012c6:	b573      	push	{r0, r1, r4, r5, r6, lr}
 80012c8:	079d      	lsls	r5, r3, #30
 80012ca:	4606      	mov	r6, r0
 80012cc:	460c      	mov	r4, r1
 80012ce:	d507      	bpl.n	80012e0 <__smakebuf_r+0x1c>
 80012d0:	f104 0347 	add.w	r3, r4, #71	; 0x47
 80012d4:	6023      	str	r3, [r4, #0]
 80012d6:	6123      	str	r3, [r4, #16]
 80012d8:	2301      	movs	r3, #1
 80012da:	6163      	str	r3, [r4, #20]
 80012dc:	b002      	add	sp, #8
 80012de:	bd70      	pop	{r4, r5, r6, pc}
 80012e0:	ab01      	add	r3, sp, #4
 80012e2:	466a      	mov	r2, sp
 80012e4:	f7ff ffca 	bl	800127c <__swhatbuf_r>
 80012e8:	9900      	ldr	r1, [sp, #0]
 80012ea:	4605      	mov	r5, r0
 80012ec:	4630      	mov	r0, r6
 80012ee:	f7ff fa73 	bl	80007d8 <_malloc_r>
 80012f2:	b948      	cbnz	r0, 8001308 <__smakebuf_r+0x44>
 80012f4:	f9b4 300c 	ldrsh.w	r3, [r4, #12]
 80012f8:	059a      	lsls	r2, r3, #22
 80012fa:	d4ef      	bmi.n	80012dc <__smakebuf_r+0x18>
 80012fc:	f023 0303 	bic.w	r3, r3, #3
 8001300:	f043 0302 	orr.w	r3, r3, #2
 8001304:	81a3      	strh	r3, [r4, #12]
 8001306:	e7e3      	b.n	80012d0 <__smakebuf_r+0xc>
 8001308:	4b0d      	ldr	r3, [pc, #52]	; (8001340 <__smakebuf_r+0x7c>)
 800130a:	62b3      	str	r3, [r6, #40]	; 0x28
 800130c:	89a3      	ldrh	r3, [r4, #12]
 800130e:	6020      	str	r0, [r4, #0]
 8001310:	f043 0380 	orr.w	r3, r3, #128	; 0x80
 8001314:	81a3      	strh	r3, [r4, #12]
 8001316:	9b00      	ldr	r3, [sp, #0]
 8001318:	6163      	str	r3, [r4, #20]
 800131a:	9b01      	ldr	r3, [sp, #4]
 800131c:	6120      	str	r0, [r4, #16]
 800131e:	b15b      	cbz	r3, 8001338 <__smakebuf_r+0x74>
 8001320:	f9b4 100e 	ldrsh.w	r1, [r4, #14]
 8001324:	4630      	mov	r0, r6
 8001326:	f000 f88d 	bl	8001444 <_isatty_r>
 800132a:	b128      	cbz	r0, 8001338 <__smakebuf_r+0x74>
 800132c:	89a3      	ldrh	r3, [r4, #12]
 800132e:	f023 0303 	bic.w	r3, r3, #3
 8001332:	f043 0301 	orr.w	r3, r3, #1
 8001336:	81a3      	strh	r3, [r4, #12]
 8001338:	89a0      	ldrh	r0, [r4, #12]
 800133a:	4305      	orrs	r5, r0
 800133c:	81a5      	strh	r5, [r4, #12]
 800133e:	e7cd      	b.n	80012dc <__smakebuf_r+0x18>
 8001340:	08000631 	.word	0x08000631

08001344 <__malloc_lock>:
 8001344:	4801      	ldr	r0, [pc, #4]	; (800134c <__malloc_lock+0x8>)
 8001346:	f7ff ba45 	b.w	80007d4 <__retarget_lock_acquire_recursive>
 800134a:	bf00      	nop
 800134c:	20000090 	.word	0x20000090

08001350 <__malloc_unlock>:
 8001350:	4801      	ldr	r0, [pc, #4]	; (8001358 <__malloc_unlock+0x8>)
 8001352:	f7ff ba40 	b.w	80007d6 <__retarget_lock_release_recursive>
 8001356:	bf00      	nop
 8001358:	20000090 	.word	0x20000090

0800135c <_free_r>:
 800135c:	b537      	push	{r0, r1, r2, r4, r5, lr}
 800135e:	2900      	cmp	r1, #0
 8001360:	d048      	beq.n	80013f4 <_free_r+0x98>
 8001362:	f851 3c04 	ldr.w	r3, [r1, #-4]
 8001366:	9001      	str	r0, [sp, #4]
 8001368:	2b00      	cmp	r3, #0
 800136a:	f1a1 0404 	sub.w	r4, r1, #4
 800136e:	bfb8      	it	lt
 8001370:	18e4      	addlt	r4, r4, r3
 8001372:	f7ff ffe7 	bl	8001344 <__malloc_lock>
 8001376:	4a20      	ldr	r2, [pc, #128]	; (80013f8 <_free_r+0x9c>)
 8001378:	9801      	ldr	r0, [sp, #4]
 800137a:	6813      	ldr	r3, [r2, #0]
 800137c:	4615      	mov	r5, r2
 800137e:	b933      	cbnz	r3, 800138e <_free_r+0x32>
 8001380:	6063      	str	r3, [r4, #4]
 8001382:	6014      	str	r4, [r2, #0]
 8001384:	b003      	add	sp, #12
 8001386:	e8bd 4030 	ldmia.w	sp!, {r4, r5, lr}
 800138a:	f7ff bfe1 	b.w	8001350 <__malloc_unlock>
 800138e:	42a3      	cmp	r3, r4
 8001390:	d90b      	bls.n	80013aa <_free_r+0x4e>
 8001392:	6821      	ldr	r1, [r4, #0]
 8001394:	1862      	adds	r2, r4, r1
 8001396:	4293      	cmp	r3, r2
 8001398:	bf04      	itt	eq
 800139a:	681a      	ldreq	r2, [r3, #0]
 800139c:	685b      	ldreq	r3, [r3, #4]
 800139e:	6063      	str	r3, [r4, #4]
 80013a0:	bf04      	itt	eq
 80013a2:	1852      	addeq	r2, r2, r1
 80013a4:	6022      	streq	r2, [r4, #0]
 80013a6:	602c      	str	r4, [r5, #0]
 80013a8:	e7ec      	b.n	8001384 <_free_r+0x28>
 80013aa:	461a      	mov	r2, r3
 80013ac:	685b      	ldr	r3, [r3, #4]
 80013ae:	b10b      	cbz	r3, 80013b4 <_free_r+0x58>
 80013b0:	42a3      	cmp	r3, r4
 80013b2:	d9fa      	bls.n	80013aa <_free_r+0x4e>
 80013b4:	6811      	ldr	r1, [r2, #0]
 80013b6:	1855      	adds	r5, r2, r1
 80013b8:	42a5      	cmp	r5, r4
 80013ba:	d10b      	bne.n	80013d4 <_free_r+0x78>
 80013bc:	6824      	ldr	r4, [r4, #0]
 80013be:	4421      	add	r1, r4
 80013c0:	1854      	adds	r4, r2, r1
 80013c2:	42a3      	cmp	r3, r4
 80013c4:	6011      	str	r1, [r2, #0]
 80013c6:	d1dd      	bne.n	8001384 <_free_r+0x28>
 80013c8:	681c      	ldr	r4, [r3, #0]
 80013ca:	685b      	ldr	r3, [r3, #4]
 80013cc:	6053      	str	r3, [r2, #4]
 80013ce:	4421      	add	r1, r4
 80013d0:	6011      	str	r1, [r2, #0]
 80013d2:	e7d7      	b.n	8001384 <_free_r+0x28>
 80013d4:	d902      	bls.n	80013dc <_free_r+0x80>
 80013d6:	230c      	movs	r3, #12
 80013d8:	6003      	str	r3, [r0, #0]
 80013da:	e7d3      	b.n	8001384 <_free_r+0x28>
 80013dc:	6825      	ldr	r5, [r4, #0]
 80013de:	1961      	adds	r1, r4, r5
 80013e0:	428b      	cmp	r3, r1
 80013e2:	bf04      	itt	eq
 80013e4:	6819      	ldreq	r1, [r3, #0]
 80013e6:	685b      	ldreq	r3, [r3, #4]
 80013e8:	6063      	str	r3, [r4, #4]
 80013ea:	bf04      	itt	eq
 80013ec:	1949      	addeq	r1, r1, r5
 80013ee:	6021      	streq	r1, [r4, #0]
 80013f0:	6054      	str	r4, [r2, #4]
 80013f2:	e7c7      	b.n	8001384 <_free_r+0x28>
 80013f4:	b003      	add	sp, #12
 80013f6:	bd30      	pop	{r4, r5, pc}
 80013f8:	20000084 	.word	0x20000084

080013fc <_read_r>:
 80013fc:	b538      	push	{r3, r4, r5, lr}
 80013fe:	4d07      	ldr	r5, [pc, #28]	; (800141c <_read_r+0x20>)
 8001400:	4604      	mov	r4, r0
 8001402:	4608      	mov	r0, r1
 8001404:	4611      	mov	r1, r2
 8001406:	2200      	movs	r2, #0
 8001408:	602a      	str	r2, [r5, #0]
 800140a:	461a      	mov	r2, r3
 800140c:	f7fe ffd5 	bl	80003ba <_read>
 8001410:	1c43      	adds	r3, r0, #1
 8001412:	d102      	bne.n	800141a <_read_r+0x1e>
 8001414:	682b      	ldr	r3, [r5, #0]
 8001416:	b103      	cbz	r3, 800141a <_read_r+0x1e>
 8001418:	6023      	str	r3, [r4, #0]
 800141a:	bd38      	pop	{r3, r4, r5, pc}
 800141c:	20000098 	.word	0x20000098

08001420 <_fstat_r>:
 8001420:	b538      	push	{r3, r4, r5, lr}
 8001422:	4d07      	ldr	r5, [pc, #28]	; (8001440 <_fstat_r+0x20>)
 8001424:	2300      	movs	r3, #0
 8001426:	4604      	mov	r4, r0
 8001428:	4608      	mov	r0, r1
 800142a:	4611      	mov	r1, r2
 800142c:	602b      	str	r3, [r5, #0]
 800142e:	f7ff f809 	bl	8000444 <_fstat>
 8001432:	1c43      	adds	r3, r0, #1
 8001434:	d102      	bne.n	800143c <_fstat_r+0x1c>
 8001436:	682b      	ldr	r3, [r5, #0]
 8001438:	b103      	cbz	r3, 800143c <_fstat_r+0x1c>
 800143a:	6023      	str	r3, [r4, #0]
 800143c:	bd38      	pop	{r3, r4, r5, pc}
 800143e:	bf00      	nop
 8001440:	20000098 	.word	0x20000098

08001444 <_isatty_r>:
 8001444:	b538      	push	{r3, r4, r5, lr}
 8001446:	4d06      	ldr	r5, [pc, #24]	; (8001460 <_isatty_r+0x1c>)
 8001448:	2300      	movs	r3, #0
 800144a:	4604      	mov	r4, r0
 800144c:	4608      	mov	r0, r1
 800144e:	602b      	str	r3, [r5, #0]
 8001450:	f7ff f808 	bl	8000464 <_isatty>
 8001454:	1c43      	adds	r3, r0, #1
 8001456:	d102      	bne.n	800145e <_isatty_r+0x1a>
 8001458:	682b      	ldr	r3, [r5, #0]
 800145a:	b103      	cbz	r3, 800145e <_isatty_r+0x1a>
 800145c:	6023      	str	r3, [r4, #0]
 800145e:	bd38      	pop	{r3, r4, r5, pc}
 8001460:	20000098 	.word	0x20000098

08001464 <_init>:
 8001464:	b5f8      	push	{r3, r4, r5, r6, r7, lr}
 8001466:	bf00      	nop
 8001468:	bcf8      	pop	{r3, r4, r5, r6, r7}
 800146a:	bc08      	pop	{r3}
 800146c:	469e      	mov	lr, r3
 800146e:	4770      	bx	lr

08001470 <_fini>:
 8001470:	b5f8      	push	{r3, r4, r5, r6, r7, lr}
 8001472:	bf00      	nop
 8001474:	bcf8      	pop	{r3, r4, r5, r6, r7}
 8001476:	bc08      	pop	{r3}
 8001478:	469e      	mov	lr, r3
 800147a:	4770      	bx	lr
